:100000000C94460018950000189500001895000003
:10001000189500001895000018950000189500002C
:10002000189500001895000018950000189500001C
:10003000189500001895000018950000189500000C
:1000400018950000189500001895000018950000FC
:1000500018950000189500001895000018950000EC
:1000600018950000189500001895000018950000DC
:1000700018950000189500000C947A371895000028
:100080001895000018950000189500008FEF8DBF9F
:10009000C0E8E8E94E2E80E18EBFD0E1FFE05F2EA0
:1000A000A89584B7082E877F84BF88E1992781BDF2
:1000B00091BDEEEFFFE0A0E0B1E088278D9331978E
:1000C000E9F780E08093980080E18093990088E1CF
:1000D00080939A00662480919A00806880939A00A9
:1000E0000E949C3881E0809345028FE787BB83EFB5
:1000F00082BB85E08093570288E08093580286E0B7
:100100008093590289E080935A0288E080935B02D1
:100110008EE080935C0289E080935D028FE08093A3
:100120005E020E942133709A80E080934E0280E04C
:10013000809353020E94572D0E944A2281E08093AF
:100140004E0285E0809353020E944A22E8EBFBE2D4
:100150000E9471370E9453325A924A9280E0A42D35
:10016000B52D8C9381E00E9464325A924A9280E0CD
:10017000A42DB52D8C9381E00E9464325A924A924C
:100180008FEAA42DB52D8C9381E00E9464325A929F
:100190004A9283E8A42DB52D8C9381E00E946432AD
:1001A0000E945823289684E00E94603278940E942E
:1001B0002D130027A0EDB1E08C9187FB0EF401E038
:1001C00041E0041711F00C941D018091D0018F774C
:1001D0008093D0010E949C38A0E5B1E03FE30E94EB
:1001E000BF320E949938ADE3B1E00E94AE37A0E57E
:1001F000B1E08C91082F0A3011F00C941B01A0E59E
:10020000B1E00E947F38082F41E0041BA1EDB1E06E
:100210000C93A0E5B1E00E947F38EA2FFB2F0091FC
:10022000D1013197E01BF0400FEFA0E5B1E00E9453
:1002300067380C94F7000E9443020091450240E1A8
:10024000040FA6E4B2E00C930027A0E3B0E08C9189
:1002500084FB0EF401E040E0041711F00C946F01F0
:1002600000914102003011F00C946A01A5E4B2E063
:10027000AD90BB24A0E3B2E0AA0CBB1CAA0DBB1D31
:100280000D911C9141E050E0040F151FAEE3B2E068
:100290000D931C93A0E4B1E0EEE3F2E00E94D237AC
:1002A000EAEEF1E70E9471370E940333A0E8BFE055
:1002B000E6E4F2E00E94D9370E94FB32EEEEF1E76D
:1002C0000E9471370E940333A0E4B1E00E94FD3226
:1002D0000E940A3381E0809341020C94720180E015
:1002E000809341020027A0E3B0E08C9187FB0EF4DD
:1002F00001E040E0041711F00C94BD0100914002B0
:10030000003011F00C94B801A5E4B2E0AD90BB242C
:10031000A0E3B2E0AA0CBB1CAA0DBB1D0D911C9161
:1003200041E050E0041B150BAEE3B2E00D931C93CB
:10033000A0E4B1E0EEE3F2E00E94D237EAEEF1E7AA
:100340000E9471370E940333A0E8BFE0E6E4F2E0C8
:100350000E94D9370E94FB32EEEEF1E70E9471371E
:100360000E940333A0E4B1E00E94FD320E940A33F0
:1003700081E0809340020C94C00180E080934002B1
:100380000027A0E3B0E08C9185FB0EF401E040E093
:10039000041711F00C94E90100914202003011F0B1
:1003A0000C94E40100914502013011F00C94DD0140
:1003B00086E0809345020C94E201809145028150D1
:1003C000809345020E942D1381E0809342020C9499
:1003D000EC0180E0809342020027A0E3B0E08C9122
:1003E00086FB0EF401E040E0041711F00C941602B5
:1003F00000914302003011F00C941102A5E4B2E028
:100400008C918F5F8C9300914502063018F011F0AB
:100410000C940C020C940F0280E0809345020E9421
:100420002D1381E0809343020C94190280E08093A5
:1004300043020027A0E3B0E08C9181FB0EF401E0C1
:1004400040E0041711F00C9438020091440200308F
:1004500011F00C943302E0EFF1E70E9471370E9433
:1004600003330E940A3381E0809344020C943B02E0
:1004700080E0809344020C94D9008091D001806880
:100480008093D0010895A0E5B1E08C91082F03324C
:1004900011F00C944D020C948102A0E5B1E08C9116
:1004A000082F0B3111F00C9457020C948102A0E537
:1004B000B1E0E8EFF1E70E9471372FEF91E00E9481
:1004C0007C34A8EDB1E00C930091D801023011F01A
:1004D0000C948102E0E5F1E00091D801A0E9B1E0DF
:1004E0000E946738A0E9B1E00E942338A2EDB1E094
:1004F0000C930091D201023011F00C9481020E9401
:1005000082020895A0E5B1E00E947F38082F42E002
:10051000041BA8EDB1E00C93A0E5B1E00E947F3888
:10052000EA2FFB2F0091D8013197E01BF0400FEF2D
:10053000A0E9B1E00E946738A0E9B1E0EEEEF1E792
:100540000E9471372FEF91E00E947C34A8EDB1E05A
:100550000C930091D801003018F011F00C94B20205
:100560000C94B70280E08093D7010C94C10281E023
:100570008093D701A0E9B1E00E947F38A8EDB1E0F7
:100580008C93E0E9F1E00091D801A0E4B1E00E9491
:100590006738A0E4B1E00E942338A3EDB1E00D93E9
:1005A0001C930091D701003011F00C942C13A0E99A
:1005B000B1E00E947F38082F4091D801041BA7EDBD
:1005C000B1E00C93A0E9B1E00E947F38EA2FFB2F45
:1005D0000091D7013197E01BF0400FEFA0E4B1E0AC
:1005E0000E946738A0E4B1E00E942338A5EDB1E095
:1005F0000D931C93A3EDB1E00D911C91033050E0DD
:10060000150711F00C948704E0E4F1E0ABEDB1E0E4
:1006100013E021E001E033270E942D375A924A92DD
:10062000EBEDF1E0A42DB52D0E94553885E10E9437
:1006300064325A924A9288E1A42DB52D8C9381E0C0
:100640000E9464325A924A9285E5A42DB52D8C936E
:1006500081E00E9464325A924A9281E0A42DB52D25
:100660008C9381E00E9464325A924A9281E0A42DD8
:10067000B52D8C9381E00E9464325A924A9281E0B7
:10068000A42DB52D8C9381E00E9464325A924A9237
:1006900080E090E0A42DB52D8D939C9382E00E9484
:1006A00064325A924A928FEF9FEFA42DB52D8D930D
:1006B0009C9382E00E9464320E94982A60968EE1A8
:1006C0000E946032A5E1B2E00D911C91A7E1B2E079
:1006D0004D915C91040F151FA9E1B2E00D931C939D
:1006E000A9E1B2E00D911C9142E050E00E947C3201
:1006F000A9E1B2E04D935C93A9E1B2E00D911C91A8
:10070000013050E0150780E00CF481E08F93A9E1FF
:10071000B2E00D911C910F3F5FEF150780E014F0E0
:1007200009F081E09F918923882311F40C949E03A2
:1007300080E090E0A9E1B2E08D939C93ADE1B2E05E
:10074000E9E1F2E00E94D237EDE1F2E0A0E8BFE09B
:100750000E945538E0E8FFE0ADE1B2E014E021E0AE
:1007600002E031E00E942D37EDE1F2E006E0ADE17C
:10077000B2E00E946738ABE1B2E04D915C91A9E133
:10078000B2E00D911C91041715071CF011F00C94A8
:10079000CB030C942704A9E1B2E08D919C91ABE1CD
:1007A000B2E08D939C935A924A92EDE1F2E0A42D2F
:1007B000B52D0E94553885E10E9464325A924A92C2
:1007C00087E8A42DB52D8C9381E00E9464325A9263
:1007D0004A928AE3A42DB52D8C9381E00E94643265
:1007E0005A924A9281E0A42DB52D8C9381E00E940B
:1007F00064325A924A9281E0A42DB52D8C9381E007
:100800000E9464325A924A9281E0A42DB52D8C93B5
:1008100081E00E9464325A924A9280E090E0A42DD6
:10082000B52D8D939C9382E00E9464325A924A9235
:100830008FEF9FEFA42DB52D8D939C9382E00E94A6
:1008400064320E94982A60968EE10E946032ADE187
:10085000B2E00E94B632EAEFF1E70E9471370E94DF
:1008600039345A924A92EDE1F2E0A42DB52D0E945E
:10087000553885E10E9464325A924A9282E3A42D4F
:10088000B52D8C9381E00E9464325A924A9286E29E
:10089000A42DB52D8C9381E00E9464325A924A9225
:1008A00081E0A42DB52D8C9381E00E9464325A9290
:1008B0004A9281E0A42DB52D8C9381E00E94643290
:1008C0005A924A9281E0A42DB52D8C9381E00E942A
:1008D00064325A924A9280E090E0A42DB52D8D9317
:1008E0009C9382E00E9464325A924A928FEF9FEF6B
:1008F000A42DB52D8D939C9382E00E9464320E94BA
:10090000982A60968EE10E9460320C942C13073076
:1009100050E0150711F00C94DB05A5EDB1E00D9149
:100920001C91003050E015070CF402C00C94B10487
:1009300080E080930502A5EDB1E00D911C914FEF91
:100940005FEF0E942F34A5EDB1E00D931C93009151
:10095000D50145E00E946F38A6E0B2E00C930C94FC
:10096000BC0480E0809306020091D50145E00E941E
:100970006F38A5E0B2E00C93A5EDB1E00D911C91AC
:10098000003A50E015071CF011F00C94C9040C94C7
:10099000D10480E098EFA7E0B2E08D939C930C9493
:1009A000D70480EE97E0A7E0B2E08D939C9300918E
:1009B0000602043218F011F00C94E0040C94E304E5
:1009C00084E2809306020AE540910602040FA6E045
:1009D000B2E00C935A924A9284E6A42DB52D8C93E2
:1009E00081E00E9464325A924A928AE5A42DB52D84
:1009F0008C9381E00E9464325A924A9289E6A42D37
:100A0000B52D8C9381E00E9464325A924A92809173
:100A10000602A42DB52D8C9381E00E9464325A9277
:100A20004A92A7E0B2E08D919C91A42DB52D8D93B3
:100A30009C9382E00E9464320E947D262A9686E082
:100A40000E9460325A924A9284E6A42DB52D8C936E
:100A500081E00E9464325A924A9280910602A42D4B
:100A6000B52D8C9381E00E9464325A924A9289E6B5
:100A7000A42DB52D8C9381E00E9464325A924A9243
:100A80008EE7A42DB52D8C9381E00E9464325A929A
:100A90004A928FEF9FEFA42DB52D8D939C9382E00A
:100AA0000E9464320E947D262A9686E00E9460326F
:100AB00000910502043218F011F00C9461050C94B9
:100AC000640584E2809305020AE540910502041B57
:100AD000A5E0B2E00C935A924A9284E6A42DB52D7B
:100AE0008C9381E00E9464325A924A92809105026E
:100AF000A42DB52D8C9381E00E9464325A924A92C3
:100B000089E6A42DB52D8C9381E00E9464325A921F
:100B10004A928AE5A42DB52D8C9381E00E9464321F
:100B20005A924A92A7E0B2E08D919C91A42DB52DE6
:100B30008D939C9382E00E9464320E947D262A96C7
:100B400086E00E9460325A924A9284E6A42DB52D26
:100B50008C9381E00E9464325A924A9285E3A42DDC
:100B6000B52D8C9381E00E9464325A924A9289E6B4
:100B7000A42DB52D8C9381E00E9464325A924A9242
:100B800080910502A42DB52D8C9381E00E946432E2
:100B90005A924A928FEF9FEFA42DB52D8D939C937F
:100BA00082E00E9464320E947D262A9686E00E949E
:100BB00060320C942C13083050E0150711F00C949F
:100BC0003107A5EDB1E00D911C91003050E0150703
:100BD0001CF011F00C94EE050C94FB0580E0809362
:100BE00006020091D50145E00E946F38A5E0B2E011
:100BF0000C930C94120680E080930502A5EDB1E001
:100C00000D911C914FEF5FEF0E942F34A5EDB1E0E5
:100C10000D931C930091D50145E00E946F38A6E02A
:100C2000B2E00C93A5EDB1E00D911C91003A50E0BB
:100C300015071CF011F00C941F060C94270680E099
:100C400098EFA7E0B2E08D939C930C942D0680EE74
:100C500097E0A7E0B2E08D939C93009106020432E6
:100C600018F011F00C9436060C94390684E2809347
:100C700006020AE540910602040FA6E0B2E00C93DA
:100C80005A924A9286E4A42DB52D8C9381E00E945D
:100C900064325A924A928AE5A42DB52D8C9381E054
:100CA0000E9464325A924A928BE4A42DB52D8C9303
:100CB00081E00E9464325A924A9280910602A42DE9
:100CC000B52D8C9381E00E9464325A924A92A7E03B
:100CD000B2E08D919C91A42DB52D8D939C9382E0D3
:100CE0000E9464320E947D262A9686E00E9460322D
:100CF0005A924A9286E4A42DB52D8C9381E00E94ED
:100D000064325A924A9280910602A42DB52D8C939A
:100D100081E00E9464325A924A928BE4A42DB52D50
:100D20008C9381E00E9464325A924A928EE7A42DFD
:100D3000B52D8C9381E00E9464325A924A928FEFD3
:100D40009FEFA42DB52D8D939C9382E00E94643279
:100D50000E947D262A9686E00E946032009105025C
:100D6000043218F011F00C94B7060C94BA0684E221
:100D7000809305020AE540910502041BA5E0B2E05C
:100D80000C935A924A9286E4A42DB52D8C9381E05F
:100D90000E9464325A924A9280910502A42DB52D88
:100DA0008C9381E00E9464325A924A928BE4A42D83
:100DB000B52D8C9381E00E9464325A924A928AE562
:100DC000A42DB52D8C9381E00E9464325A924A92F0
:100DD000A7E0B2E08D919C91A42DB52D8D939C93AD
:100DE00082E00E9464320E947D262A9686E00E945C
:100DF00060325A924A9286E4A42DB52D8C9381E0FC
:100E00000E9464325A924A9285E3A42DB52D8C93A8
:100E100081E00E9464325A924A928BE4A42DB52D4F
:100E20008C9381E00E9464325A924A92809105022A
:100E3000A42DB52D8C9381E00E9464325A924A927F
:100E40008FEF9FEFA42DB52D8D939C9382E00E9490
:100E500064320E947D262A9686E00E9460320C94BD
:100E60002C13093050E0150711F00C948F08A5EDF4
:100E7000B1E08D919C91A5E1B2E08D939C93A5ED9D
:100E8000B1E00D911C91003050E015071CF011F0FD
:100E90000C944C070C94590780E080930602009153
:100EA000D50145E00E946F38A5E0B2E00C930C94A8
:100EB000700780E080930502A5EDB1E00D911C91D3
:100EC0004FEF5FEF0E942F34A5EDB1E00D931C931F
:100ED0000091D50145E00E946F38A6E0B2E00C9386
:100EE000A5EDB1E00D911C91003A50E015071CF002
:100EF00011F00C947D070C94850780E098EFA7E033
:100F0000B2E08D939C930C948B078FE190E0A7E067
:100F1000B2E08D939C9300910602043218F011F018
:100F20000C9494070C94970784E2809306020AE5D8
:100F300040910602040FA6E0B2E00C935A924A9246
:100F40008BE4A42DB52D8C9381E00E9464325A92DB
:100F50004A928AE5A42DB52D8C9381E00E946432DB
:100F60005A924A9280E5A42DB52D8C9381E00E947F
:100F700064325A924A9280910602A42DB52D8C9328
:100F800081E00E9464325A924A92A7E0B2E08D91C9
:100F90009C91A42DB52D8D939C9382E00E94643288
:100FA0000E947D262A9686E00E9460325A924A92DA
:100FB0008BE4A42DB52D8C9381E00E9464325A926B
:100FC0004A9280910602A42DB52D8C9381E00E9457
:100FD00064325A924A9280E5A42DB52D8C9381E01B
:100FE0000E9464325A924A928EE7A42DB52D8C93BA
:100FF00081E00E9464325A924A928FEF9FEFA42DB3
:10100000B52D8D939C9382E00E9464320E947D26D0
:101010002A9686E00E94603200910502043218F0A0
:1010200011F00C9415080C94180884E280930502C2
:101030000AE540910502041BA5E0B2E00C935A9228
:101040004A928BE4A42DB52D8C9381E00E946432EA
:101050005A924A9280910502A42DB52D8C9381E07D
:101060000E9464325A924A9280E5A42DB52D8C9349
:1010700081E00E9464325A924A928AE5A42DB52DED
:101080008C9381E00E9464325A924A92A7E0B2E0C7
:101090008D919C91A42DB52D8D939C9382E00E94FF
:1010A00064320E947D262A9686E00E9460325A921F
:1010B0004A928BE4A42DB52D8C9381E00E9464327A
:1010C0005A924A9285E3A42DB52D8C9381E00E941B
:1010D00064325A924A9280E5A42DB52D8C9381E01A
:1010E0000E9464325A924A9280910502A42DB52D35
:1010F0008C9381E00E9464325A924A928FEF9FEF64
:10110000A42DB52D8D939C9382E00E9464320E94A1
:101110007D262A9686E00E9460320C942C130A30B9
:1011200050E0150711F00C94EB09A5EDB1E08D919D
:101130009C91A7E1B2E08D939C93A5EDB1E00D9158
:101140001C91003050E015070CF402C00C94C1084B
:1011500080E080930502A5EDB1E00D911C914FEF69
:101160005FEF0E942F34A5EDB1E00D931C93009129
:10117000D50145E00E946F38A6E0B2E00C930C94D4
:10118000CC0880E0809306020091D50145E00E94E2
:101190006F38A5E0B2E00C93A5EDB1E00D911C9184
:1011A000003A50E015071CF011F00C94D9080C948B
:1011B000E10880E098EFA7E0B2E08D939C930C9457
:1011C000E7088FE190E0A7E0B2E08D939C93009157
:1011D0000602043218F011F00C94F0080C94F30895
:1011E00084E2809306020AE540910602040FA6E01D
:1011F000B2E00C935A924A928FE5A42DB52D8C93B0
:1012000081E00E9464325A924A928AE5A42DB52D5B
:101210008C9381E00E9464325A924A9284E6A42D13
:10122000B52D8C9381E00E9464325A924A9280914B
:101230000602A42DB52D8C9381E00E9464325A924F
:101240004A92A7E0B2E08D919C91A42DB52D8D938B
:101250009C9382E00E9464320E947D262A9686E05A
:101260000E9460325A924A928FE5A42DB52D8C933C
:1012700081E00E9464325A924A9280910602A42D23
:10128000B52D8C9381E00E9464325A924A9284E692
:10129000A42DB52D8C9381E00E9464325A924A921B
:1012A0008EE7A42DB52D8C9381E00E9464325A9272
:1012B0004A928FEF9FEFA42DB52D8D939C9382E0E2
:1012C0000E9464320E947D262A9686E00E94603247
:1012D00000910502043218F011F00C9471090C947D
:1012E000740984E2809305020AE540910502041B1B
:1012F000A5E0B2E00C935A924A928FE5A42DB52D49
:101300008C9381E00E9464325A924A928091050245
:10131000A42DB52D8C9381E00E9464325A924A929A
:1013200084E6A42DB52D8C9381E00E9464325A92FC
:101330004A928AE5A42DB52D8C9381E00E946432F7
:101340005A924A92A7E0B2E08D919C91A42DB52DBE
:101350008D939C9382E00E9464320E947D262A969F
:1013600086E00E9460325A924A928FE5A42DB52DF4
:101370008C9381E00E9464325A924A9285E3A42DB4
:10138000B52D8C9381E00E9464325A924A9284E691
:10139000A42DB52D8C9381E00E9464325A924A921A
:1013A00080910502A42DB52D8C9381E00E946432BA
:1013B0005A924A928FEF9FEFA42DB52D8D939C9357
:1013C00082E00E9464320E947D262A9686E00E9476
:1013D00060320C942C130B3050E0150711F00C9474
:1013E000970CE0EFF1E0A0E4B1E00E94873811F43F
:1013F0000C94950CE0E4F1E0A0EFB1E00E945538C8
:101400005A924A92A42DB52DE0E0F2E70E9471377E
:101410000E94393485E10E9464325A924A928AE0ED
:10142000A42DB52D8C9381E00E9464325A924A9289
:1014300089E1A42DB52D8C9381E00E9464325A92EB
:101440004A9281E0A42DB52D8C9381E00E946432F4
:101450005A924A9281E0A42DB52D8C9381E00E948E
:1014600064325A924A9281E0A42DB52D8C9381E08A
:101470000E9464325A924A928FEF9FEFA42DB52DAD
:101480008D939C9382E00E9464325A924A928FEF2D
:101490009FEFA42DB52D8D939C9382E00E94643222
:1014A0000E94982A60968EE10E946032A5EDB1E01C
:1014B0000D911C910A3050E0150711F00C94B80AF8
:1014C0005A924A92A42DB52DE6E1F2E70E947137B7
:1014D0000E94393482E10E9464325A924A928AE030
:1014E000A42DB52D8C9381E00E9464325A924A92C9
:1014F00089E1A42DB52D8C9381E00E9464325A922B
:101500004A9281E0A42DB52D8C9381E00E94643233
:101510005A924A9281E0A42DB52D8C9381E00E94CD
:1015200064325A924A9281E0A42DB52D8C9381E0C9
:101530000E9464325A924A9280E098EFA42DB52D11
:101540008D939C9382E00E9464325A924A928FEF6C
:101550009FEFA42DB52D8D939C9382E00E94643261
:101560000E94982A60968BE10E9460320C94950C40
:101570000B3050E0150711F00C94160B5A924A925A
:10158000A42DB52DE8E2F2E70E9471370E943934AC
:1015900083E10E9464325A924A928AE0A42DB52DCA
:1015A0008C9381E00E9464325A924A9289E1A42D80
:1015B000B52D8C9381E00E9464325A924A9281E068
:1015C000A42DB52D8C9381E00E9464325A924A92E8
:1015D00081E0A42DB52D8C9381E00E9464325A9253
:1015E0004A9281E0A42DB52D8C9381E00E94643253
:1015F0005A924A9280E098EFA42DB52D8D939C933A
:1016000082E00E9464325A924A928FEF9FEFA42D9B
:10161000B52D8D939C9382E00E9464320E94982A9B
:1016200060968CE10E9460320C94950C0C3050E076
:10163000150711F00C94740B5A924A92A42DB52DF3
:10164000ECE3F2E70E9471370E94393482E10E9494
:1016500064325A924A928AE0A42DB52D8C9381E08F
:101660000E9464325A924A9289E1A42DB52D8C933E
:1016700081E00E9464325A924A9281E0A42DB52DF5
:101680008C9381E00E9464325A924A9281E0A42DA8
:10169000B52D8C9381E00E9464325A924A9281E087
:1016A000A42DB52D8C9381E00E9464325A924A9207
:1016B00080E098EFA42DB52D8D939C9382E00E943D
:1016C00064325A924A928FEF9FEFA42DB52D8D93DD
:1016D0009C9382E00E9464320E94982A60968BE17B
:1016E0000E9460320C94950C0D3050E0150711F0FB
:1016F0000C94D20B5A924A92A42DB52DEEE4F2E747
:101700000E9471370E94393483E10E9464325A92F8
:101710004A928AE0A42DB52D8C9381E00E94643218
:101720005A924A9289E1A42DB52D8C9381E00E94B2
:1017300064325A924A9281E0A42DB52D8C9381E0B7
:101740000E9464325A924A9281E0A42DB52D8C9366
:1017500081E00E9464325A924A9281E0A42DB52D14
:101760008C9381E00E9464325A924A9280E098EF12
:10177000A42DB52D8D939C9382E00E9464325A92E1
:101780004A928FEF9FEFA42DB52D8D939C9382E00D
:101790000E9464320E94982A60968CE10E94603216
:1017A0000C94950C0E3050E0150711F00C94300C91
:1017B0005A924A92A42DB52DE2E6F2E70E947137C3
:1017C0000E94393485E10E9464325A924A928AE03A
:1017D000A42DB52D8C9381E00E9464325A924A92D6
:1017E00089E1A42DB52D8C9381E00E9464325A9238
:1017F0004A9281E0A42DB52D8C9381E00E94643241
:101800005A924A9281E0A42DB52D8C9381E00E94DA
:1018100064325A924A9281E0A42DB52D8C9381E0D6
:101820000E9464325A924A9280E098EFA42DB52D1E
:101830008D939C9382E00E9464325A924A928FEF79
:101840009FEFA42DB52D8D939C9382E00E9464326E
:101850000E94982A60968EE10E9460320C94950C4A
:10186000A0E4B1E0E8E7F2E70E9471370E94853812
:1018700011F00C94410C80E090E0ABE1B2E08D936C
:101880009C935A924A92E0E4F1E0A42DB52D0E9477
:10189000553880E10E9464325A924A928AE0A42D1F
:1018A000B52D8C9381E00E9464325A924A9289E16C
:1018B000A42DB52D8C9381E00E9464325A924A92F5
:1018C00081E0A42DB52D8C9381E00E9464325A9260
:1018D0004A9281E0A42DB52D8C9381E00E94643260
:1018E0005A924A9281E0A42DB52D8C9381E00E94FA
:1018F00064325A924A9280E090E0A42DB52D8D93E7
:101900009C9382E00E9464325A924A928FEF9FEF3A
:10191000A42DB52D8D939C9382E00E9464320E9489
:10192000982A609689E10E9460320C942C130C3046
:1019300050E0150711F00C94C40DA0E4B1E00E9432
:101940003836EDE0F0E0A9E0B2E00E945A38E2EC6F
:10195000F1E70E9471370E941936E9E0F2E00E9437
:10196000EB340E948035EDE0F0E0A9E0B2E00E94A7
:101970005A38E9E0F2E00E94EB34E6ECF1E70E942D
:1019800071370E9419360E94223681E008F480E007
:101990008F93E9E0F2E00E94EB34EAECF1E70E9479
:1019A00071370E9419360E94223681E010F009F04A
:1019B00080E09F918923882311F40C94E70C80E048
:1019C00098EFA7E0B2E08D939C930C94490DE9E069
:1019D000F2E00E94EB34EAECF1E70E9471370E94DA
:1019E00019360E94223681E008F480E08F93E9E006
:1019F000F2E00E94EB34EEECF1E70E9471370E94B6
:101A000019360E94223681E010F009F080E09F91A3
:101A10008923882311F40C94150D86EC9CEFA7E024
:101A2000B2E08D939C930C94490DE9E0F2E00E94A2
:101A3000EB34EEECF1E70E9471370E9419360E94F8
:101A4000223681E008F480E08F93E9E0F2E00E9422
:101A5000EB34E2EDF1E70E9471370E9419360E94E3
:101A6000223681E010F009F080E09F9189238823DD
:101A700011F40C94430D80EE97E0A7E0B2E08D9353
:101A80009C930C94490D80E090E0A7E0B2E08D9328
:101A90009C93A0E4B1E0E9E0F2E00E94EB340E9404
:101AA0004A33E0E4F1E004E0A0E4B1E00E946738EA
:101AB000E0E4F1E0ABEDB1E012E0222701E03327F2
:101AC0000E942D37ABEDB1E00E94B632E0E8F2E7BC
:101AD0000E9471370E9439345A924A92EBEDF1E03C
:101AE000A42DB52D0E94553885E10E9464325A928A
:101AF0004A9288E1A42DB52D8C9381E00E94643236
:101B00005A924A9284E3A42DB52D8C9381E00E94D1
:101B100064325A924A9281E0A42DB52D8C9381E0D3
:101B20000E9464325A924A9281E0A42DB52D8C9382
:101B300081E00E9464325A924A9281E0A42DB52D30
:101B40008C9381E00E9464325A924A92A7E0B2E0FC
:101B50008D919C91A42DB52D8D939C9382E00E9434
:101B600064325A924A928FEF9FEFA42DB52D8D9338
:101B70009C9382E00E9464320E94982A60968EE1D3
:101B80000E9460320C942C130F3050E0150711F0B6
:101B90000C94100FA0E4B1E00E943836EDE0F0E0C4
:101BA000ADE0B2E00E945A38E6EDF1E70E947137ED
:101BB0000E941936EDE0F2E00E94EB340E94B2354B
:101BC000EDE0F0E0ADE0B2E00E945A38EAEDF1E776
:101BD0000E9471370E941936EDE0F2E00E94EB346A
:101BE0000E948035EDE0F0E0ADE0B2E00E945A38AE
:101BF000EDE0F2E00E94EB34E6ECF1E70E94713791
:101C00000E9419360E94223681E008F480E08F930A
:101C1000EDE0F2E00E94EB34EEEDF1E70E94713767
:101C20000E9419360E94223681E010F009F080E00F
:101C30009F918923882311F40C94260E80EE97E05F
:101C4000A7E0B2E08D939C930C94880EEDE0F2E057
:101C50000E94EB34EEEDF1E70E9471370E941936D5
:101C60000E94223681E008F480E08F93EDE0F2E0FC
:101C70000E94EB34E2EEF1E70E9471370E941936C0
:101C80000E94223681E010F009F080E09F918923C4
:101C9000882311F40C94540E86EC9CEFA7E0B2E07C
:101CA0008D939C930C94880EEDE0F2E00E94EB344F
:101CB000EEECF1E70E9471370E9419360E9422363D
:101CC00081E008F480E08F93EDE0F2E00E94EB34D5
:101CD000E6EEF1E70E9471370E9419360E94223623
:101CE00081E010F009F080E09F918923882311F4AE
:101CF0000C94820E80E098EFA7E0B2E08D939C9365
:101D00000C94880E80EE97E0A7E0B2E08D939C9350
:101D1000EDE0F2E00E94A238EDE0F0E00E94AD3488
:101D2000A9EDB1E0EE0C000FE794DD92EC92A0E497
:101D3000B1E0E9EDF1E00E94D237E0E4F1E004E047
:101D4000A0E4B1E00E946738E0E4F1E0ABEDB1E07F
:101D500013E021E000E033270E942D37ABEDB1E026
:101D60000E94B632E2E8F2E70E9471370E943934ED
:101D70005A924A92EBEDF1E0A42DB52D0E94553810
:101D800085E10E9464325A924A9288E1A42DB52DD1
:101D90008C9381E00E9464325A924A928AE6A42D82
:101DA000B52D8C9381E00E9464325A924A9281E070
:101DB000A42DB52D8C9381E00E9464325A924A92F0
:101DC00081E0A42DB52D8C9381E00E9464325A925B
:101DD0004A9281E0A42DB52D8C9381E00E9464325B
:101DE0005A924A92A7E0B2E08D919C91A42DB52D14
:101DF0008D939C9382E00E9464325A924A928FEFB4
:101E00009FEFA42DB52D8D939C9382E00E946432A8
:101E10000E94982A60968EE10E9460320C942C13E6
:101E2000003150E0150711F00C945C10A0E4B1E013
:101E30000E943836EDE0F0E0A1E1B2E00E945A38AD
:101E4000E6EDF1E70E9471370E941936E1E1F2E018
:101E50000E94EB340E94B235EDE0F0E0A1E1B2E087
:101E60000E945A38EAEDF1E70E9471370E94193654
:101E7000E1E1F2E00E94EB340E948035EDE0F0E019
:101E8000A1E1B2E00E945A38E1E1F2E00E94EB34B5
:101E9000E6ECF1E70E9471370E9419360E94223663
:101EA00081E008F480E08F93E1E1F2E00E94EB34FE
:101EB000EEEDF1E70E9471370E9419360E9422363A
:101EC00081E010F009F080E09F918923882311F4CC
:101ED0000C94720F80EE97E0A7E0B2E08D939C9394
:101EE0000C94D40FE1E1F2E00E94EB34EEEDF1E767
:101EF0000E9471370E9419360E94223681E008F450
:101F000080E08F93E1E1F2E00E94EB34E2EEF1E752
:101F10000E9471370E9419360E94223681E010F02B
:101F200009F080E09F918923882311F40C94A00F7D
:101F300086EC9CEFA7E0B2E08D939C930C94D40FB9
:101F4000E1E1F2E00E94EB34EEECF1E70E94713740
:101F50000E9419360E94223681E008F480E08F93B7
:101F6000E1E1F2E00E94EB34E6EEF1E70E94713726
:101F70000E9419360E94223681E010F009F080E0BC
:101F80009F918923882311F40C94CE0F80E098EF61
:101F9000A7E0B2E08D939C930C94D40F80EE97E071
:101FA000A7E0B2E08D939C93E1E1F2E00E94A238B9
:101FB000EDE0F0E00E94AD34A9EDB1E0EE0C000FD1
:101FC000E794DD92EC92A0E4B1E0E9EDF1E00E944B
:101FD000D237E0E4F1E004E0A0E4B1E00E94673829
:101FE000E0E4F1E0ABEDB1E013E021E000E0332705
:101FF0000E942D37ABEDB1E00E94B632E2E8F2E785
:102000000E9471370E9439345A924A92EBEDF1E006
:10201000A42DB52D0E94553885E10E9464325A9254
:102020004A9288E1A42DB52D8C9381E00E94643200
:102030005A924A9284E7A42DB52D8C9381E00E9498
:1020400064325A924A9281E0A42DB52D8C9381E09E
:102050000E9464325A924A9281E0A42DB52D8C934D
:1020600081E00E9464325A924A9281E0A42DB52DFB
:102070008C9381E00E9464325A924A92A7E0B2E0C7
:102080008D919C91A42DB52D8D939C9382E00E94FF
:1020900064325A924A928FEF9FEFA42DB52D8D9303
:1020A0009C9382E00E9464320E94982A60968EE19E
:1020B0000E9460320C942C13013150E0150711F08E
:1020C0000C94D410A5EDB1E08D919C91A2E3B2E007
:1020D0008D939C93ABEDB1E0E4E8F2E70E94713799
:1020E0000E943934E0E4F1E0ABEDB1E00E94B63299
:1020F00013E021E001E033270E942D375A924A92E3
:10210000EBEDF1E0A42DB52D0E94553885E10E943C
:1021100064325A924A9289E7A42DB52D8C9381E0BE
:102120000E9464325A924A9288E4A42DB52D8C9371
:1021300081E00E9464325A924A9281E0A42DB52D2A
:102140008C9381E00E9464325A924A9281E0A42DDD
:10215000B52D8C9381E00E9464325A924A9281E0BC
:10216000A42DB52D8C9381E00E9464325A924A923C
:1021700080E090E0A42DB52D8D939C9382E00E9489
:1021800064325A924A928FEF9FEFA42DB52D8D9312
:102190009C9382E00E9464320E94982A60968EE1AD
:1021A0000E9460320C942C13023150E0150711F09C
:1021B0000C944C11A5EDB1E08D919C91A4E3B2E09B
:1021C0008D939C93ABEDB1E0EAE8F2E70E947137A2
:1021D0000E943934E0E4F1E0ABEDB1E00E94B632A8
:1021E00013E021E001E033270E942D375A924A92F2
:1021F000EBEDF1E0A42DB52D0E94553885E10E944C
:1022000064325A924A9289E7A42DB52D8C9381E0CD
:102210000E9464325A924A9282E5A42DB52D8C9385
:1022200081E00E9464325A924A9281E0A42DB52D39
:102230008C9381E00E9464325A924A9281E0A42DEC
:10224000B52D8C9381E00E9464325A924A9281E0CB
:10225000A42DB52D8C9381E00E9464325A924A924B
:1022600080E090E0A42DB52D8D939C9382E00E9498
:1022700064325A924A928FEF9FEFA42DB52D8D9321
:102280009C9382E00E9464320E94982A60968EE1BC
:102290000E9460320C942C13033150E0150711F0AA
:1022A0000C94C411A5EDB1E08D919C91A6E3B2E030
:1022B0008D939C93ABEDB1E0E0E9F2E70E947137BA
:1022C0000E943934E0E4F1E0ABEDB1E00E94B632B7
:1022D00013E021E001E033270E942D375A924A9201
:1022E000EBEDF1E0A42DB52D0E94553885E10E945B
:1022F00064325A924A9289E7A42DB52D8C9381E0DD
:102300000E9464325A924A928CE5A42DB52D8C938A
:1023100081E00E9464325A924A9281E0A42DB52D48
:102320008C9381E00E9464325A924A9281E0A42DFB
:10233000B52D8C9381E00E9464325A924A9281E0DA
:10234000A42DB52D8C9381E00E9464325A924A925A
:1023500080E090E0A42DB52D8D939C9382E00E94A7
:1023600064325A924A928FEF9FEFA42DB52D8D9330
:102370009C9382E00E9464320E94982A60968EE1CB
:102380000E9460320C942C13043150E0150711F0B8
:102390000C943C12A5EDB1E08D919C91A8E3B2E0C4
:1023A0008D939C93ABEDB1E0E6E9F2E70E947137C3
:1023B0000E943934E0E4F1E0ABEDB1E00E94B632C6
:1023C00013E021E001E033270E942D375A924A9210
:1023D000EBEDF1E0A42DB52D0E94553885E10E946A
:1023E00064325A924A9289E7A42DB52D8C9381E0EC
:1023F0000E9464325A924A9286E6A42DB52D8C939F
:1024000081E00E9464325A924A9281E0A42DB52D57
:102410008C9381E00E9464325A924A9281E0A42D0A
:10242000B52D8C9381E00E9464325A924A9281E0E9
:10243000A42DB52D8C9381E00E9464325A924A9269
:1024400080E090E0A42DB52D8D939C9382E00E94B6
:1024500064325A924A928FEF9FEFA42DB52D8D933F
:102460009C9382E00E9464320E94982A60968EE1DA
:102470000E9460320C942C13053150E0150711F0C6
:102480000C94B412A5EDB1E08D919C91AAE3B2E059
:102490008D939C93ABEDB1E0ECE9F2E70E947137CC
:1024A0000E943934E0E4F1E0ABEDB1E00E94B632D5
:1024B00013E021E001E033270E942D375A924A921F
:1024C000EBEDF1E0A42DB52D0E94553885E10E9479
:1024D00064325A924A9289E7A42DB52D8C9381E0FB
:1024E0000E9464325A924A9280E7A42DB52D8C93B3
:1024F00081E00E9464325A924A9281E0A42DB52D67
:102500008C9381E00E9464325A924A9281E0A42D19
:10251000B52D8C9381E00E9464325A924A9281E0F8
:10252000A42DB52D8C9381E00E9464325A924A9278
:1025300080E090E0A42DB52D8D939C9382E00E94C5
:1025400064325A924A928FEF9FEFA42DB52D8D934E
:102550009C9382E00E9464320E94982A60968EE1E9
:102560000E9460320C942C13063150E0150711F0D4
:102570000C942C13A5EDB1E08D919C91ACE3B2E0ED
:102580008D939C93ABEDB1E0E2EAF2E70E947137E4
:102590000E943934E0E4F1E0ABEDB1E00E94B632E4
:1025A00013E021E001E033270E942D375A924A922E
:1025B000EBEDF1E0A42DB52D0E94553885E10E9488
:1025C00064325A924A9289E7A42DB52D8C9381E00A
:1025D0000E9464325A924A928AE7A42DB52D8C93B8
:1025E00081E00E9464325A924A9281E0A42DB52D76
:1025F0008C9381E00E9464325A924A9281E0A42D29
:10260000B52D8C9381E00E9464325A924A9281E007
:10261000A42DB52D8C9381E00E9464325A924A9287
:1026200080E090E0A42DB52D8D939C9382E00E94D4
:1026300064325A924A928FEF9FEFA42DB52D8D935D
:102640009C9382E00E9464320E94982A60968EE1F8
:102650000E9460320C942C130895009145020130C1
:1026600011F00C946A135A924A9285E7A42DB52D65
:102670008C9381E00E9464325A924A9288E4A42D9D
:10268000B52D8C9381E00E9464325A924A9288E779
:10269000A42DB52D8C9381E00E9464325A924A9207
:1026A0008EE4A42DB52D8C9381E00E9464325A9261
:1026B0004A9280E090E0A42DB52D8D939C9382E00A
:1026C0000E9464320E947D262A9686E00E94603233
:1026D0000C949F135A924A9285E7A42DB52D8C93A2
:1026E00081E00E9464325A924A9288E4A42DB52D6A
:1026F0008C9381E00E9464325A924A9288E7A42D1A
:10270000B52D8C9381E00E9464325A924A928EE4F5
:10271000A42DB52D8C9381E00E9464325A924A9286
:102720008FEF9FEFA42DB52D8D939C9382E00E9497
:1027300064320E947D262A9686E00E9460320091D3
:102740004502023011F00C94DC135A924A9285E74C
:10275000A42DB52D8C9381E00E9464325A924A9246
:1027600082E5A42DB52D8C9381E00E9464325A92AB
:102770004A9288E7A42DB52D8C9381E00E946432A3
:102780005A924A9288E5A42DB52D8C9381E00E943F
:1027900064325A924A9280E090E0A42DB52D8D9338
:1027A0009C9382E00E9464320E947D262A9686E0F5
:1027B0000E9460320C9411145A924A9285E7A42D1B
:1027C000B52D8C9381E00E9464325A924A9282E540
:1027D000A42DB52D8C9381E00E9464325A924A92C6
:1027E00088E7A42DB52D8C9381E00E9464325A9223
:1027F0004A9288E5A42DB52D8C9381E00E94643225
:102800005A924A928FEF9FEFA42DB52D8D939C93F2
:1028100082E00E9464320E947D262A9686E00E9411
:10282000603200914502033011F00C944E145A921C
:102830004A9285E7A42DB52D8C9381E00E946432E5
:102840005A924A928CE5A42DB52D8C9381E00E947A
:1028500064325A924A9288E7A42DB52D8C9381E078
:102860000E9464325A924A9282E6A42DB52D8C932E
:1028700081E00E9464325A924A9280E090E0A42D56
:10288000B52D8D939C9382E00E9464320E947D2638
:102890002A9686E00E9460320C9483145A924A92DF
:1028A00085E7A42DB52D8C9381E00E9464325A9265
:1028B0004A928CE5A42DB52D8C9381E00E94643260
:1028C0005A924A9288E7A42DB52D8C9381E00E94FC
:1028D00064325A924A9282E6A42DB52D8C9381E0FF
:1028E0000E9464325A924A928FEF9FEFA42DB52D29
:1028F0008D939C9382E00E9464320E947D262A96EA
:1029000086E00E94603200914502043011F00C9480
:10291000C0145A924A9285E7A42DB52D8C9381E07C
:102920000E9464325A924A9286E6A42DB52D8C9369
:1029300081E00E9464325A924A9288E7A42DB52D14
:102940008C9381E00E9464325A924A928CE6A42DC4
:10295000B52D8C9381E00E9464325A924A9280E0B5
:1029600090E0A42DB52D8D939C9382E00E9464325B
:102970000E947D262A9686E00E9460320C94F5140F
:102980005A924A9285E7A42DB52D8C9381E00E943E
:1029900064325A924A9286E6A42DB52D8C9381E03A
:1029A0000E9464325A924A9288E7A42DB52D8C93E6
:1029B00081E00E9464325A924A928CE6A42DB52D91
:1029C0008C9381E00E9464325A924A928FEF9FEF7B
:1029D000A42DB52D8D939C9382E00E9464320E94B9
:1029E0007D262A9686E00E946032009145020530DD
:1029F00011F00C9432155A924A9285E7A42DB52D08
:102A00008C9381E00E9464325A924A9280E7A42D0E
:102A1000B52D8C9381E00E9464325A924A9288E7E5
:102A2000A42DB52D8C9381E00E9464325A924A9273
:102A300086E7A42DB52D8C9381E00E9464325A92D2
:102A40004A9280E090E0A42DB52D8D939C9382E076
:102A50000E9464320E947D262A9686E00E9460329F
:102A60000C9467155A924A9285E7A42DB52D8C9344
:102A700081E00E9464325A924A9280E7A42DB52DDB
:102A80008C9381E00E9464325A924A9288E7A42D86
:102A9000B52D8C9381E00E9464325A924A9286E767
:102AA000A42DB52D8C9381E00E9464325A924A92F3
:102AB0008FEF9FEFA42DB52D8D939C9382E00E9404
:102AC00064320E947D262A9686E00E946032009140
:102AD0004502063011F00C94A4155A924A9285E7EB
:102AE000A42DB52D8C9381E00E9464325A924A92B3
:102AF0008AE7A42DB52D8C9381E00E9464325A920E
:102B00004A9288E7A42DB52D8C9381E00E9464320F
:102B10005A924A9280E8A42DB52D8C9381E00E94B0
:102B200064325A924A9280E090E0A42DB52D8D93A4
:102B30009C9382E00E9464320E947D262A9686E061
:102B40000E9460320C94D9155A924A9285E7A42DBE
:102B5000B52D8C9381E00E9464325A924A928AE7A2
:102B6000A42DB52D8C9381E00E9464325A924A9232
:102B700088E7A42DB52D8C9381E00E9464325A928F
:102B80004A9280E8A42DB52D8C9381E00E94643296
:102B90005A924A928FEF9FEFA42DB52D8D939C935F
:102BA00082E00E9464320E947D262A9686E00E947E
:102BB00060320895F894FFCF5C8B8585008B858506
:102BC000008B8585008B8585008B8585008B855BDB
:102BD000390E39380F380F38390E390E39380F3869
:102BE0000F38390E390E39380F38390E39380F3859
:102BF000390E39FBFB78AFD8D800D9D8D800D9DF47
:102C0000E6EDE6E0DFD8D800D9D8D800AE0E3939E5
:102C1000000E393900380F38393900380F39383952
:102C2000380F383939000E390E3939000E3939006C
:102C30000E390E3939000EFBFB788BD8AEAE00D9B9
:102C4000BCFBFB05EEDFAEAFD87E396939380F38F3
:102C50000F3809380F3F633908390E3909380F38F2
:102C60003933380F38390E3933380F3839FBFB0E0A
:102C7000F4F402FBFB01F4F402FBFB02F4F401FBAD
:102C8000FB02F4EDE7F4FBFB1EF4EDED00E7FBFBCC
:102C900000F4F400E7E700F4FBFB2385D8D9DEF469
:102CA000FBFB07D1DFD8AEAE0069FBFB0039323940
:102CB0000E3939003801FBFB00703938390E63CA10
:102CC000C4390E390E39330E390E390E39380FFB2F
:102CD000FB0CE0DFD3D8D3DFE7EDE0D9D2D9D900C0
:102CE000DFEEFBE6D9D3D9E0FBEDE0D2D9D2E7FBAA
:102CF000FB1CE7DFD3D2D201F4F400E0D2D201DF33
:102D0000FBFB2385D8AEEEFBFB05D1FBFB02DFD935
:102D1000AE62FBF50E390E3939000E3908F4FB703E
:102D2000380F380F62FBFB00390F38390E39380F76
:102D3000383938390938FBFB0CE0D2D203E0EDD941
:102D4000D2D203E0FAE7D2D201E0F4DFD2D202E637
:102D5000FBFB1BF4D9D2D202D9FBEDD2D202E0FBAD
:102D6000FB2385D8EDFBFB02D1EDE6EDFBFB03ED8C
:102D7000AE8469FBD13839C4FBFB00C43907FBFBC7
:102D800000696900CBCA93CBFBFB00CA6339CBFB5C
:102D9000FB009A3938CBCA93FB9AFBFB0DE0D2D2E9
:102DA00002E0FBEDD9D2D201D3F4FBFB00DFD2E08D
:102DB000FAFBEDD3D2D201E7FBFB1CE7D2D202DF54
:102DC000FBF5EDE6E7F4FBFB24B5AEFBD1FBFB0125
:102DD000E6AED8AEDFFBFB03DFA862FBFB0032CA26
:102DE000FB9A99FBCB07D0FBC4FBFB006938CAFBFD
:102DF000FB00A062FBFB00CAFAFBC432FBFB0270C3
:102E0000FBFB0DEDD3D2A8D2DFF4FBAFD2D202B6DA
:102E1000FBF4B6D2EDFBFB00F4D9D2D201E6FBF411
:102E2000E7EDF4FBFB04F4EDE7EDF4FBFB04F4ED5C
:102E3000E7EDF4FBFB01F4DFD2D201E0FAFBFB008B
:102E4000D1F4EDED00FBFB02F4F400E7EDED00FB47
:102E5000FB1A85E0FBFB02F4AFD8D9AED9F4FBFB3B
:102E600002ED8469FBF439FBFB006968FBFB00326F
:102E7000FBFB029A380862FBFB003869FBFA086228
:102E8000FBFB0037FBFB009A3839FBFB0DF4D9D272
:102E9000D201D3EDF5D2D203D8F5EDD2D9F4FBFBB4
:102EA00000EEAED2D201E6EED9D2D200E0F4FBFBC6
:102EB00002E6D9D2D200D9DFEEFBFB02E0D9D2D2B2
:102EC00000D3DFEEFBFB01D9A8D2D200E0CBFBEDB3
:102ED000E0D9D3D2FBFB01F4E0D8D2D200D3E0F4A6
:102EE000FBFB1885ECFBFB07D1FBFB01D1FBEDAE37
:102EF00062FBFB0068FBFB00F5FBF4FB38F4FBFB1B
:102F000002390F62FBFB000E93FBCB3938FBFB0051
:102F100038FBFB00630F38FBFB0EE7D2D201A8E0C1
:102F2000E6D2D204E0E000D2E0FBFB01F4D9D2D239
:102F300000A8D9D900D2D202E0FBFB01E0D2D20036
:102F4000D9E7D2D200D9EDFBF5E6D2D200D3ECD945
:102F5000D2D9EDFBFB00D9D2D201DFFBEDD2D202F8
:102F6000A8F4FBF4D9D2D200E0E6D2D200E0F4FB20
:102F7000FB1785EDFBFB08FAFBFB02F47E68FBD137
:102F800031FBFB000E0869690007FBFB0099F5FBAC
:102F90009A3862FBFB006962FBFB003893FBD1624D
:102FA000FBFB0039380FFBFB0EF4D2D205AFD2D2B7
:102FB00005EDFBFB01EED8D2D201DFE7D9D2D20179
:102FC000E0FBFB00EDD2D201D9EDD9D2D200E0FB7B
:102FD000EDD2D201D9EDD3D2D200E6FBF4D9D2D2D0
:102FE00001E0FBF4E0D2D201D8F5FBE0D2D201E05F
:102FF000E6D3D2D200EDFBFB1785EDFBFB0DF4AE63
:1030000062FBFB003299FBFB02C407CBFB6968FB48
:10301000FB003F38FBFB0162CAFBFB027031FBFB8C
:103020000039390038FBFB0FE0D2D203D3EDD9D2FF
:10303000D200A8D2D200D8CBFBFB01F4D9D2D20166
:10304000E6D1E0D2A8D2DFFBFB00E0D2A8D2D201C9
:10305000A8D2D200DFFBE6D2D200A8D2D201A8D2F9
:10306000D9FBCBDFD2D201B5FBFB00E6D2D202F511
:10307000FAAFD2D201A8D2D202E7FBFB17AFECFB2A
:10308000FB00D1FBFAC3E7ECEDED02E7EDED00BC90
:10309000A8389370080800629A99690F31699939C4
:1030A0003269996908629A9A000F07939A9A0039CF
:1030B0003808996F390E39FBFB0FEDD2D203E6FBCE
:1030C000E7D2D203E7FBFB02EED9D2D201E7FBDF66
:1030D000D2D201D3FBFB00DFD2D201D9E0E6E60079
:1030E000E7C4FBDFD2D201D9E6E600E7E6F4FBF461
:1030F000D9D2D3D2E0FBFB00B6D2D202FBEED9D2BA
:10310000D201DFE7E6E600EDFAFBFB1785B6FBFB35
:1031100003D8D800AED2AED2AEAE00D8A8D884388C
:103120000E393839380E390E3939010E39380F3821
:103130000F38390E0E0038390E380E38390E330E6E
:1031400039380FFBFB0FFAB6D2D201A8EDFBFAD942
:10315000D2D201D9EDFBFB02F3D3A8D2D200E6FB19
:10316000E0D2D202FBFB00E7D2D201D9FBFB01FA8D
:10317000FBFB00E7D2D201D8F5FBFB01D1FBFB0042
:10318000D9D2D201E0F4FBE7D2D202F4F400DFD2CC
:10319000D201E0FBFB00D1F5FBFB1885D8FBFB035C
:1031A000BDD8AFD8DFF4F403DF7E390F380F380F06
:1031B0003938390E390E3939000E393900380F389F
:1031C0003939010F390F3939000E39390038390FC3
:1031D00038FBFB10E0D8D2D200D9FBFB01E0D2D201
:1031E00001E0F4FBFB02EDD2D202E0FBE0D2D2011F
:1031F000D8F5FBEED2D202E6EEEDE0EEFBEDAFD27B
:10320000D200D3E6F4EDE0EEFBF4D9D2A8D2DFF59C
:10321000FAE0D2D200A8D9F4D1E7D2D201D9EDEEAA
:10322000EDE0FAFBFB178BD8BDFAFBFB02FAEDEEE3
:10323000FBFB03FAD9AE083839383939000E330FA1
:103240003839380F38390E39083939000E330E380D
:103250003932380F38390E390F3839FBFB10F4D9B1
:10326000D2D3E6FBFB01F4AFD2D200C3FBFB02D109
:10327000E0D2D203EDD9A8D2D201B6FBFB00C3D273
:10328000D201A8D2D200B5F4FBFB00EDD3D2D2001C
:10329000A8D2D200DFF4FBE0D2D203E7EED2D20311
:1032A000DFF5FAE0D2D200A8D2D201E6F5FBFB1797
:1032B000B5D8D800F4FBFB09CBDFAE849ACBCAC5E6
:1032C000CACA00CBCACA00C5CAC5CACBC4CBCACBFE
:1032D000CACA00CBCACBC4CBCACBC4CBCAC5CACA24
:1032E00000C5CAFBFB10D1EDD9E0F4FBFB02E6D927
:1032F000E6FBFB04E6E0D9D900AFE0EEE6DFD3D988
:10330000DFEDFBFB00FAEEE0D9D900DFE7F5FBFBD0
:1033100002EDDFD9D900DFE7F4FBFB00EDDFD3D806
:10332000D9DFC3F4E0DFD3D9DFE7FBFB00F4E7DF4D
:10333000D3D9E0EDFBFB19E0AFD8AEEDD1FBFB0339
:10334000D1FBFB00F4DFAED8AEC4FBFB34F4FAFBD8
:10335000FB04F4F5FBFB05F4F402FBFB01F5F4F4CC
:1033600000FBFB05F4F400F5FBFB06F4F400F5FBB1
:10337000FB02D1FBF4F401F5FBFB01F4F401F5D100
:10338000FBFB01D1F5FAF4FBFB1BDFD8AED9D8E08B
:10339000F4FAFBFB02F4BCD9D8D9AEAFCAFBFB9A56
:1033A000E6AFD8AED8AED2AFDFB5DFB5D8D800AE75
:1033B000D8AED884C4FBFB9AC38C628C8C00628B21
:1033C0008C628C8C008B628C8C00628C8C0062CA4C
:1033D000FBFBFFFBFBFFFBFBFFFBFBFFFBFBFFFB29
:1033E000FBFFFBFBFFFBFBFFFBFBFFFBFBFFFBFB19
:1033F000FFFBFBFFFBFBFFFBFBFFFBFBFFFBFBFF05
:10340000FBFBFFFBFBFFFBFBFFFBFBCD9269926825
:1034100093689269689269689269686800936268C3
:1034200069688C69686800636868006962686968CF
:1034300062696868006368680069626869686269EF
:103440006862FBFB0A696862696868006368680013
:1034500069626869686269686800636868006962CF
:1034600068696862696868006368680069626869B9
:103470006862696862FBFB27D1FBFB1B6893FBFB5F
:103480002F6869FBFB066292FBFB286869FBFB4225
:1034900093FBFB3362FBFB0468FBFB2C62FBFB40F2
:1034A00068FBFB3568FBFB0268FBFB2E68FBFB221D
:1034B000F5FBFB1993FBFB05C59A9A00949A9A00B9
:1034C000C4FBFB2968FBFB0069FBFB3062FBFB21B3
:1034D000FAFBFB01FAF5D1FBFB00F4D1FBFB0F6813
:1034E000FBFB03CB9A9A00CBFBFB00CBC46A94FB9B
:1034F000FB2893FBFB0092FBFB3093FBFB04D1FB0F
:10350000FB14D1FBFB02D1FBFB1993FBFB049A9448
:10351000FBCAC4CA9A9398649AFBFB288C69FBFB8C
:103520003268FBFB2FCAFBFB0968FBFB049A9BCBB1
:10353000FACAC3CACA009A649AFBFB286992FBFBC9
:103540003293FBFB17D1FAFBFB01F5FBFB1C93FB52
:10355000FB04EDCB9AC59B9ACAC5CB9968FBFB28A7
:103560009269FBFB3268FBFB18F5FBFB18CAFBFBFF
:103570000568FBFB04C9FAF5CA9A9A00C59AC3BC50
:1035800062FBFB286992FBFB3269FBFB1CFAFBFB2D
:103590000CF5FBFB0D93FBFB04F3F4F400C2B48BBE
:1035A0008A8A00BB8B62FBFB289269FBFB3262FBC1
:1035B000FB20F5FBFB01F5FBFB1468FBFB04CAF4E5
:1035C000F3BC8A8BB48BBB8B92FBFB286992FBFB11
:1035D0003293FBFB21D1FBFB02FAFBFB01FAFBFB65
:1035E0000E93FBFB049ACAF3EC8A8BB48BBB9269F3
:1035F000FBFB289269FBFB3268FBFB14FAFBFB0A1E
:10360000FAFBFB03CBFBFB01D1FBFB0D68FBFB04CF
:103610009B9AC4C3BBBB00929200933363FBFB280D
:103620006992FBFB3293FBFB14CBFBFB05D1FBFB4D
:1036300016F5FBFB0393FBFB0494959B393409338C
:1036400033013263FBFB289269FBFB3268FBFB1BF7
:10365000F5FBFB11D0FBF5FBFB01D0FBFB0368FB8B
:10366000FB049B706A640933393333000963FBFB45
:10367000286992FBFB3293FBFB2CF5FBFB0C93FBC5
:10368000FB046A956A640933330009330963FBFB61
:10369000289269FBFB3268FBFB1CFAFBFB1C68FBF6
:1036A000FB049B6A643933093333010863FBFB284D
:1036B0006992FBFB3293FBFB17FAD1FBFB04F5FB92
:1036C000FB1993FBFB04946B6433092D3909330216
:1036D00063FBFB289269FBFB3268FBFB18F5FBFBE5
:1036E00009D1FBFB00F5FBFB1168FBFB046A6A00D8
:1036F000643A3309333300090269FBFB286992FB02
:10370000FB3293FBFB1FD1FAFBFB00F5FAFBFB023C
:10371000FAFBFB0F93FBFB049B643A330933330042
:1037200009330263FBFB289269FBFB3262FBFB045B
:10373000FAFBFB24D1FBFB05D0FBFB0568FBFB047C
:103740006A6439333300023933030869FBFB2869A3
:1037500092FBFB3293FBFB04D1FBFB15F5FBFB0C4F
:10376000F5FBFB00FAF5FBFB01F5FBFB0693FBFB0E
:1037700003CB6A64330933330263CAFBFB2792FB32
:1037800069FBFB3268FBFB08CAFBFB3168FBFB05EE
:103790009A39333300396369CBFBFB2869FB92FB11
:1037A000FB3269FBFB15CBFBFB02D1FBFB0AD1FB18
:1037B000FB1393FBFB3592FBFB0069FBFB3292FB97
:1037C000FB17FAFBFB02FAFBFB10D1FBFB0C68FBBF
:1037D000FB3369FBFB0192FBFB3269FBFB20F5FB32
:1037E000FB03F5FBFB0DD0FBFB069368FBFB2F698E
:1037F00092FBFB0269FBFB3292FBFB1AF5FBFB051C
:10380000D1FBFB04FAFBFB09F5FBFB09926992680B
:10381000926992920169926893686392699263686F
:103820009368636869629368696269688D686968AA
:1038300063689362696869629368636893FBFB04D9
:1038400092FBFB3269FBFB20FAFBFB01FAFBFB045A
:10385000F5FBFB139263689369926969019269931E
:10386000689392696893689392699293929392692C
:103870009293929392699293929392699293929374
:103880006893929368FBFB0469FBFB3268FBFB1EA9
:10389000D1FBFB10FAFBFB0B6869FBFB00FAC3C30F
:1038A00000FBFB04ED98CAFBFB219368FBFB029233
:1038B000FBFB3293FBFB14FAF5FBFB0BF5FBFB0464
:1038C000D1FBFB03F5FBFB0B68FBFB02CA9992CA19
:1038D000FBFB03998CCAFBFB2393FBFB0169FBFBFE
:1038E0003268FBFB18D1FBFB03F5FBFB0BFAFBFB80
:1038F00003D1FBFB0868FBFB03F5988BC4FBFB02C1
:10390000FA9392FAFBFB2468FBFB0092FBFB3293D9
:10391000FBFB14D1FBFB02FAFBFB09D1FBFB14639D
:10392000FBFB05CA92C3CACA02C399C3FBFB269319
:10393000FB69FBFB3262FBFB0BD0FBFB0BF5FBFBDC
:103940000DF5FBFB1092FBFB05CA9992C3CAC3CAD3
:103950009398CAFBFB2668FB92FBFB3293FBFB2D83
:10396000F5FBFB03F5FBFAFBFB0368FBFB079992F6
:10397000CAFBFB01CA93C3CAFBFB269369FBFB325C
:1039800068FBFB05FAFBFB18D0FBFB0BD1FBFB0A2A
:1039900093FBFB04CACA00C3CAC3CAFBFB00CACA62
:1039A00002C4CAF4C993FBFB226893FBFB3293FB6E
:1039B000FB1CD1FBFB01F5FBFB01FAF5FBFB08FA55
:1039C000FBFB02D1FBFB0368FBFB02D1FBF4CAF457
:1039D000FBD0C4CAFBCAC9FBFB00CAC399C3C3005E
:1039E000FBFB229368FBFB3268FBFB07D1FBFB0B65
:1039F000F5FBFB11FAFBFB0F93FBC3C300CAFAF5FF
:103A0000C3CAFBFB00F5C3CAF4C3CAFBFB00CA92DE
:103A100098C4FAFBFB226893FBFB3293FBFB14FA7E
:103A2000FBFB03FAF5FBFB09D1FBFB0CF5FBFB02EF
:103A300068FB679298C3C999CAFBFB01999900FA80
:103A400099C4FBF4CA99CAFBFB249368FBFB326858
:103A5000FBFB31F5FBFB0793FBCAC399926299CA42
:103A6000F4FBFB00C3999398C3C9CAFBC4CAFBFB10
:103A7000246992FBFB3269FBFB08FAFBFB0AD1FBD2
:103A8000FB12F5FBFB03D1FBFB0868FBFB01F4C356
:103A900093CAF4CA99C398939893C3CAF4FBCAC350
:103AA000FBFB249269FBFB3292FBFB03D0FBFB1375
:103AB000D1FBFB10D1FBFB0C93FBFB02CAC3FBFB4E
:103AC00000CACA019262926299CAFBFB00C3CAFB98
:103AD000FB246992FBFB3269FBFB0BD1FBFB08F576
:103AE000FBFB05FAF5FBD1FBF5FBFB06FAFBFB0440
:103AF000FAFBFB0568FBFB02CBC3D0FBFB01CA92C0
:103B000061379299C3CACA0099C3CAFBFB23926961
:103B1000FBFB3262FBFB26FAFBFB05F5FBFB0A9382
:103B2000FBFB02CAC3FBFB00FAC4C39962620099A3
:103B3000F4FBCAC3929200C3CAFBFB226992FBFB4F
:103B40003293FBFB13F5FBFB00FAFBFB01F5FBFBE0
:103B500008D1FBF5FBFB0AD1FBFB0468FBFB00D1A2
:103B6000FBCA99F5CAC3CAFAC399F499CAF5D1C375
:103B7000CACA00C3CAFBFB229269FBFB3268FBFB8B
:103B800003F5FBFB01D1FBFB13D1FBFB15F5FBFBA5
:103B90000369FBFB02CAC3C300CACA00FBF599CA8A
:103BA000FA99CAFBFAC4D0FBFB256992FBFB32935E
:103BB000FBFB09FAFBFB0EFAFBFB05FAFBFB16927B
:103BC000FBFB01F4999299CAFBFB01C3CAF5CAC475
:103BD000F4CACA00FBFB269269FBFB3268FBFB03BD
:103BE000FAFBFB0ED1FBFB13D1FBFB03FAF5FBFB4E
:103BF0000769FBCAC9C29299C3CAFBFACACA00FACA
:103C0000FBD0C399CAFBFB01F5FBFB236992FBFBCD
:103C10003293FBFB2AFAFBFB02D1FBFB03FAFBFB13
:103C20000392FBC98C92CAFBCAC3CACA00C4CAFBAE
:103C3000FB00CA929200FBFB289269FBFB3268FBF7
:103C4000FB03D1FBFB0DFAFBFB02D1FBFB05F5FBF4
:103C5000FB01F5FBFB05F5FBFB0C69FBCAC3CAF4D2
:103C6000FBCAC4C3999399C3C4CA9293CAFBFB27E6
:103C70006992FBFB3293FBFB16F5FBFB01F5FBFBAB
:103C800004D1FBFB1868FBCBFACBCACA01A0929205
:103C900000C3CAC9CAC49299F4FBFB2592FB69FB15
:103CA000FB3262FBFB07F5FBFB01D1FBFB11FAFBCF
:103CB000FB06F5FBFB09D1FBFB0593CAF4CACA005E
:103CC000F4CBFAC39299C4CAFBCACA00C399FBFBDE
:103CD0002669FB92FBFB3269FBFB07FAFBFB01FA4F
:103CE000FBFB05F5FBFB07D1FBFB05FAFBFB0BF52B
:103CF000FBFB0793CACA00CBCACA00CB9962C3D0E8
:103D0000FBCAFBFB00F4D1F4FBFB00CAFBFB2192D6
:103D1000FBFB0069FBFB3292FBFB16FAFBFB02FA92
:103D2000FBFB0AD1FBFB12D093FBCAF4CACA009278
:103D300091CAFBF5FBFAD1FBFB2669FBFB0192FB69
:103D4000FB3269FBFB2CFAD1FBF5FBFAFBFB0B9278
:103D500069FBFB2F9368FBFB0269FBFB3292FBFBC9
:103D600014D1FBFB05F5FBFB01F5FBFB1E926992F1
:103D7000696893626968639263686269626869628C
:103D800068696268696268696268696269686269CB
:103D9000686368680063686962686962696893FB60
:103DA000FB0492FBFB3269FBFB23D1F5FBFB04F523
:103DB000FBFB136992699392936992939293689330
:103DC0009300929393009293930092939300929313
:103DD0009300929393009293929393009293929371
:103DE00093009293929393009293929368FBFB04B7
:103DF00069FBFB3292FBFB1AD1FBFB05FAFBFB10C4
:103E0000F4FBFB076893FBFB2F9368FBFB0292FB21
:103E1000FB3269FBFB16F5FBFB0EFAFBFB07D1FB44
:103E2000FB01D1FBFB0668FBFB019993999399CAAF
:103E3000FBFB2A93FBFB0169FBFB3292FBFB3D681A
:103E4000FBFB0231696900686399FBFB2B68FBFB94
:103E50000092FBFB3269FBFB13F5FBFAFBFB02FA5A
:103E6000FBFB01D1FBFB06D1F5FBFB1193FBFB0335
:103E70003893C5F5D0C4FBFB2C93FB69FBFB329256
:103E8000FBFB0AD1FBFB0FF5FBFAFBFB0BD1FBFBAA
:103E900000FAFBF5FBFB0868FBFB03626899D1CBDA
:103EA000C4FBFB2C68FB92FBFB3269FBFB14D1FBD0
:103EB000FB09F5FBFB08FAFBFB0D93FBFB0468C455
:103EC000CBF5CB99FBFB2D9369FBFB3262FBFB032C
:103ED000FAFBFB00D1FBFB10D1FBFB1F68FBFB04D3
:103EE000629AC4D1CAC4FBFB2D6893FBFB3293FBDF
:103EF000FB08FAFBFB0DF5FBFB07D1FAF5FBFB0515
:103F0000F5FBFB04FAFBF5FBFB0393FBFB04626987
:103F100099F5CA9AFBFB2D9368FBFB3268FBFB3BD0
:103F200068FBFB0468C5CBD1CAC4FBFB2D6893FBBF
:103F3000FB3293FBFB04D1FBFB0BFAFBFB1AD1FB1F
:103F4000FB02D1FBFB0493FBFB046299C4F5CA9A04
:103F5000FBFB2D9368FBFB3268FBFB04F5FBFB05C9
:103F6000FAFBFB05F5FBFB01FAFBFB0DF4D1FBFBB8
:103F700004F5FBFB0868FBFB04689AC4D1CAC4FBC8
:103F8000FB2D6992FBFB3293FBFB04FAFBFB04D194
:103F9000FBFB03F5FBFB08D1F5FBFB1B93FBFB04D1
:103FA00062939AD1C499FBFB2D8C69FBFB3268FBB1
:103FB000FB12D1FBFB01D1FBFB07FAF5FBFB1768FA
:103FC000FBFB04629AC4F5CA99FBFB07D1FBFB23F8
:103FD0006992FBFB3269FBFB1CFAFBFB01D1FBFB8B
:103FE00001D1FBFB06FAFBFB02FAFBFB0693FBFB92
:103FF00004629A9A00CBCB0093FBFB2D9269FBFBEA
:104000003262FBFB04D1FBFB12F5FBFB19F5FBFB5A
:104010000368FBFB0462999900FB9A99FBFB2D69ED
:1040200092FBFB3293FBFB25F4FBFB03F5FBD1FB7F
:10403000FB0B93FBFB046293C5D1C499FBFB2D9250
:1040400069FBFB3268FBFB04FAFBFB02D0FBFB04C1
:10405000FAFBFB02FAFBFB18F5FBFB01D1FBFB04AF
:1040600068FBFB04629A9A00FBC499FBFB2D6992E2
:10407000FBFB3293FBFB0DD1FBFB04F5FBFB12D1E9
:10408000FBFB0F93FBFB0462999AD1C499FBFB2DB8
:104090009269FBFB3268FBFB05F5FBFB13D1F5FBDB
:1040A000FB01F5FBFB13FAFBFB0268FBFB04629AC6
:1040B000C4FBC499FBFB2D6992FBFB3293D1FBFB44
:1040C00004D1FBFB07F5FBFB04D1FBFB10FAFBFB68
:1040D0000F93FBFB04689399CBCB00629A999A9952
:1040E000C39A9999019A999900CAFBFB209269FB9E
:1040F000FB3262FBFB12D1FBFB07FAFBFB03FAFB73
:10410000FB04F5FBFB04D0FBFB02F5FBFB0368FBA8
:10411000FB046399C5D1CAC49AC49A9A01C49AC4CB
:104120009AC49A939300FBFB206992FBFB3299FBA4
:10413000FB05FAFBFB10FAFBFB05D1FBFB01CBFBFC
:10414000FB1593FBFB03629ACAF5FBCBFBCAFBF59D
:10415000FBCBFBFB00CBFBFB009399FBFB1F92FB14
:10416000FB0069FBFB3068FBFB19F5FBFB15F5FB5E
:10417000FB0968FBFB0362999ACBFBFB0ACB6999AD
:10418000FBFB1F69FBFB0092FBFB3093FBFB15F570
:10419000FBFB16F5FBFB05D1FBFB0593FBFB026963
:1041A0009AC4CAC4CAC4A0C4C400A0C49AC49AC44D
:1041B000C4006993FBFB1E92FBFB0269FBFB2E68AC
:1041C000FBFB28FAFBFB02D1FBFAFBFB0E68FBFBB7
:1041D00001623738380362383762376238613837FE
:1041E00031C3FBFB1D69FBFB0492FBFB2C69FBFB52
:1041F0001DD1FBF5FBFB01F5FBFB10FAFBFB09698D
:1042000092FBFB2F9368FBFB066968FBFB28699216
:10421000FBFB24FAFBFB12F5FBFB0969926992692F
:1042200092688D68936893689368936893686992BD
:104230006968629368680063686800936268696887
:104240006293686800636868009362686992636853
:10425000FBFB0A9362696893626968936269689379
:104260006269689362696893626968936269689336
:1042700062696893626968936269689362FBFB0490
:10428000FAFBFB15FAFBFB0CF5FBD1FBF5FBFB0482
:10429000D1FBFB0800000006000C00130019001FF2
:1042A00001400146014C01530159015F02A002A6E1
:1042B00002AC02B302B902BF04000406040C0413EA
:1042C0000419041F05400546054C05530559055FB3
:1042D00006A006A606AC06B306B906BF07E007E6C9
:1042E00007EC07F307F907FF30003006300C3013F6
:1042F0003019301F31403146314C31533159315F23
:1043000032A032A632AC32B332B932BF34003406F6
:10431000340C34133419341F35403546354C35537D
:104320003559355F36A036A636AC36B336B936BF0A
:1043300037E037E637EC37F337F937FF60006006D0
:10434000600C60136019601F61406146614C6153ED
:104350006159615F62A062A662AC62B362B962BF7A
:1043600064006406640C64136419641F6540654648
:10437000654C65536559655F66A066A666AC66B315
:1043800066B966BF67E067E667EC67F367F967FFE2
:1043900098009806980C98139819981F9940994678
:1043A000994C99539959995F9AA09AA69AAC9AB345
:1043B0009AB99ABF9C009C069C0C9C139C199C1F4C
:1043C0009D409D469D4C9D539D599D5F9EA09EA6E0
:1043D0009EAC9EB39EB99EBF9FE09FE69FEC9FF36D
:1043E0009FF99FFFC800C806C80CC813C819C81F8A
:1043F000C940C946C94CC953C959C95FCAA0CAA650
:10440000CAACCAB3CAB9CABFCC00CC06CC0CCC1358
:10441000CC19CC1FCD40CD46CD4CCD53CD59CD5F21
:10442000CEA0CEA6CEACCEB3CEB9CEBFCFE0CFE637
:10443000CFECCFF3CFF9CFFFF800F806F80CF81364
:10444000F819F81FF940F946F94CF953F959F95F91
:10445000FAA0FAA6FAACFAB3FAB9FABFFC00FC0665
:10446000FC0CFC13FC19FC1FFD40FD46FD4CFD53EC
:10447000FD59FD5FFEA0FEA6FEACFEB3FEB9FEBF79
:10448000FFE0FFE6FFECFFF3FFF9FFFF0000000095
:104490000000000081E00E94443382E00E94443327
:1044A00080914E02AA81BB818C9380E080934E0262
:1044B00080E08093470280E08093490283E8809304
:1044C00048028FEA80934A020E94A7228FEF8093CE
:1044D0005F028FEF809360028FEF809361028FEF16
:1044E000809362028FEF809363028FEF8093640268
:1044F0008FEF809365028FEF8093660281E090E0FA
:10450000A881B9818D939C93A881B9810D911C914B
:10451000003B56E1150718F011F00C949B2298E02F
:10452000AFE5B2E00E941733A881B9810E946832DA
:1045300010F40C948422C59AAA81BB818C9180933B
:104540004E0283E0481A8827580A249608958CE082
:1045500090E0AFEBB3E08D939C938FEE80935F027E
:1045600088E08093600288E18093610282E1809319
:10457000630285E18093650283E18093670286E1AF
:104580008093690200914E02003011F00C94CD220C
:1045900080E0809362020C944223023011F00C946C
:1045A000F22283E08093620203E840914702041BF9
:1045B000A7E4B2E00C9303E840914802041BA8E48E
:1045C000B2E00C930FEA40914902041BA9E4B2E067
:1045D0000C930FEA40914A02041BAAE4B2E00C9348
:1045E0000C944223013011F00C941B2385E080933E
:1045F000620203E840914902041BA9E4B2E00C9373
:1046000003E840914A02041BAAE4B2E00C93009133
:1046100047028091490280934702A9E4B2E00C93DB
:104620000091480280914A0280934802AAE4B2E0D5
:104630000C930C944223033011F00C94422386E037
:10464000809362020FEA40914702041BA7E4B2E0A4
:104650000C930FEA40914802041BA8E4B2E00C93CB
:10466000009147028091490280934702A9E4B2E099
:104670000C930091480280914A0280934802AAE478
:10468000B2E00C93809147028093640280914802CB
:1046900080936602809149028093680280914A0269
:1046A00080936A02C69A0E94C22DC598C698089542
:1046B00082E00E94443382E00E94443381E00E9401
:1046C000443381E00E94443381E08093560280E0CD
:1046D00090E0A4E5B2E08D939C93AE85BF858C916C
:1046E00080934702AC85BD858C9180934902AA8551
:1046F000BB858C9180934802A885B9858C91809365
:104700004A020E94A722AA85BB850C91AE85BF856F
:104710004C91041BAA81BB810C93AA81BB818C9113
:104720008F5F8C93A885B9850C91AC85BD854C9124
:10473000041BA881B9810C93A881B9818C918F5FEA
:104740008C93AA81BB810D911127A881B9814D91CC
:1047500055270E942F34AC81BD810D931C9381E0BD
:1047600090E0AE81BF818D939C93AC81BD814D91D2
:104770005C91AE81BF810D911C910417150718F053
:1047800011F00C94D1230E94D82392E0AFE5B2E05F
:104790000E941733AE81BF810E94683210F40C94DE
:1047A000B523C59A86E0481A8827580A289608959E
:1047B00081E00E94443381E00E94443381E00E9402
:1047C000443382E00E94443382E00E9444330091EB
:1047D0005302003011F00C9401240E945932AFE5CD
:1047E000B2E00E940F360C920E9453320E9459325E
:1047F000A0E6B2E00E940F360C920E9453320C9455
:104800008B25013011F00C94B924A4E5B2E00D9190
:104810001C91003050E0150711F00C94B324009166
:104820005602013011F00C942C240E945932AFE54D
:10483000B2E00E940F360C920E9453320E9459320D
:10484000A0E6B2E00E940F360C920E94533280E044
:10485000809356020C94B124AFE5B2E08C91AA810A
:10486000BB818D9388278C9398E0AA81BB810E949D
:104870006134AA81BB810D911C91A0E6B2E04D91FB
:104880005527040F151FAA81BB810D931C930E940D
:104890005932AFE5B2E00E940F360C920E945332BB
:1048A0000E945932A0E6B2E00E940F360C920E949C
:1048B0005332AFE5B2E08C91A881B9818D938827FE
:1048C0008C9398E0A881B9810E946134A881B98154
:1048D0000D911C91A0E6B2E04D915527040F151FD4
:1048E000A881B9810D931C93AA81BB814D915C91E4
:1048F000A881B9810D911C910417150711F00C9432
:10490000B1240E945932AC81BD810E940F360C92B5
:104910000E945332AC81BD818C91A4E5B2E08D93AD
:1049200088278C9398E0A4E5B2E00E9461340E944D
:104930005932AC81BD810E940F360C920E945332D5
:10494000A4E5B2E00D911C91AC81BD814D9155273C
:10495000040F151FA4E5B2E00D931C9381E0809332
:1049600056020C94B724A4E5B2E00E946F320C9476
:104970008B25023011F00C94CA240E945932ABE40A
:10498000B2E00E940F360C920E9453320E94BA2568
:104990000C948B25033011F00C942325A4E5B2E090
:1049A0000D911C91003050E0150711F00C941D255D
:1049B00000915602013011F00C94EE240E945932FD
:1049C000ABE4B2E00E940F360C920E9453320E9478
:1049D000BA2580E0809356020C941B2580914B02EF
:1049E000AC81BD818C930E945932ABE4B2E00E944D
:1049F0000F360C920E9453320E94BA2540914B020E
:104A0000AC81BD810C91041711F00C941B250E9400
:104A10005932AC81BD810E940F360C920E945332F4
:104A2000AC81BD818C91A4E5B2E08D9388278C93F5
:104A300081E0809356020C942125A4E5B2E00E9407
:104A40006F320C948B25043011F00C9434250E94A5
:104A50005932ABE4B2E00E940F360C920E945332FE
:104A60000E9491250C948B25053011F00C948B2518
:104A7000A4E5B2E00D911C91003050E0150711F053
:104A80000C94872500915602013011F00C945825A2
:104A90000E945932ABE4B2E00E940F360C920E94A1
:104AA00053320E94912580E0809356020C94852514
:104AB00080914B02AC81BD818C930E945932ABE452
:104AC000B2E00E940F360C920E9453320E94912550
:104AD00040914B02AC81BD810C91041711F00C94F4
:104AE00085250E945932AC81BD810E940F360C92FF
:104AF0000E945332AC81BD818C91A4E5B2E08D93CC
:104B000088278C9381E0809356020C948B25A4E532
:104B1000B2E00E946F3287E0481A8827580A2A9626
:104B20000895ABE4B2E00D91112742E050E00E94FD
:104B30002F34ACE4B2E00D931C93E4E9F2E40E945C
:104B40007137ACE4B2E08D919C91AFE5B2E00E9488
:104B50001A37ACE4B2E00E946832E4E9F2E40E9461
:104B60007137ACE4B2E08D919C91A0E6B2E00E9476
:104B70001A37089581E00E94443381E00E94443353
:104B800081E00E94443380E0AC81BD818C9380E061
:104B9000AA81BB818C9380E0A881B9818C93ABE41E
:104BA000B2E08C9181FBAC81BD818C9181F98C93B9
:104BB000ABE4B2E08C9180FBAC81BD818C9180F93B
:104BC0008C93ABE4B2E08C9184FBAA81BB818C9185
:104BD00082F98C93ABE4B2E08C9183FBAA81BB8118
:104BE0008C9181F98C93ABE4B2E08C9182FBAA8129
:104BF000BB818C9180F98C93ABE4B2E08C9187FB04
:104C0000A881B9818C9182F98C93ABE4B2E08C914C
:104C100086FBA881B9818C9181F98C93ABE4B2E0D9
:104C20008C9185FBA881B9818C9180F98C93AC81A2
:104C3000BD810C914AE0049F0C92AA81BB810C912A
:104C400049E0049F0C92A881B9810C9144E0049F33
:104C50000C92AC81BD810C910E3111F00C94342674
:104C60008FE1AC81BD818C93A881B9810C910C310D
:104C700011F00C943F268FE1A881B9818C93A88113
:104C8000B9818C9180935F0293E0AFE5B2E00E941E
:104C90005934AA81BB818C9187FBAFE5B2E08C913E
:104CA00082F98C93AA81BB818C9186FBAFE5B2E03F
:104CB0008C9181F98C93AA81BB818C9185FBAFE5A6
:104CC000B2E08C9180F98C93AA81BB818C91809306
:104CD000600293E0A0E6B2E00E94593400916002C5
:104CE000AC81BD814C91040FA0E6B2E00C9383E04F
:104CF000481A8827580A2696089582E00E9444336D
:104D000082E00E94443381E00E94443381E00E94AB
:104D10004433A889B9898C9180934702AE85BF85B9
:104D20008C9180934902AC85BD858C91809348021B
:104D3000AA85BB858C9180934A020E94A722AC85EC
:104D4000BD850C91A889B9894C91041BAA81BB81AE
:104D50000C93AA81BB818C918F5F8C93AA85BB85B4
:104D60000C91AE85BF854C91041BA881B9810C9331
:104D7000A881B9818C918F5F8C93AA81BB810D91A1
:104D80001127A881B9814D9155270E942F34AC81FC
:104D9000BD810D931C93A885B9858D919C91AFE43D
:104DA000B2E08D939C930E94492D81E090E0AE810A
:104DB000BF818D939C93AC81BD814D915C91AE81FF
:104DC000BF810D911C910417150718F011F00C9478
:104DD000F52692E0AFE5B2E00E941733AE81BF81C5
:104DE0000E94683210F40C94DB26C59A86E0481ABB
:104DF0008827580A289608955A924A92AC85BD850C
:104E00008C91A42DB52D8C9381E00E9464325A922E
:104E10004A92AC85BD858C91A42DB52D8C9381E0F3
:104E20000E9464325A924A92AC85BD858C91A42D21
:104E3000B52D8C9381E00E9464325A924A92A889DF
:104E4000B9898C91A42DB52D8C9381E00E94643298
:104E50005A924A92AC85BD858C91A42DB52D8C9328
:104E600081E00E9464325A924A92AC85BD858D9150
:104E70009C91A42DB52D8D939C9382E00E94643269
:104E80000E948F282C9687E00E9460325A924A92A4
:104E9000A885B9858C91A42DB52D8C9381E00E94B5
:104EA00064325A924A92AC85BD858C91A42DB52D61
:104EB0008C9381E00E9464325A924A92AC85BD85FF
:104EC0008C91A42DB52D8C9381E00E9464325A926E
:104ED0004A92AC85BD858C91A42DB52D8C9381E033
:104EE0000E9464325A924A92AC85BD858C91A42D61
:104EF000B52D8C9381E00E9464325A924A92AC851F
:104F0000BD858D919C91A42DB52D8D939C9382E0B0
:104F10000E9464320E948F282C9687E00E946032A3
:104F20005A924A92AC85BD858C91A42DB52D8C9357
:104F300081E00E9464325A924A92A885B9858C9188
:104F4000A42DB52D8C9381E00E9464325A924A922E
:104F5000AC85BD858C91A42DB52D8C9381E00E94EC
:104F600064325A924A92AC85BD858C91A42DB52DA0
:104F70008C9381E00E9464325A924A92AC85BD853E
:104F80008C91A42DB52D8C9381E00E9464325A92AD
:104F90004A92AC85BD858D919C91A42DB52D8D93A4
:104FA0009C9382E00E9464320E948F282C9687E0B6
:104FB0000E9460325A924A92AC85BD858C91A42D94
:104FC000B52D8C9381E00E9464325A924A92AC854E
:104FD000BD858C91A42DB52D8C9381E00E94643207
:104FE0005A924A92A889B9898C91A42DB52D8C9397
:104FF00081E00E9464325A924A92AC85BD858C91C0
:10500000A42DB52D8C9381E00E9464325A924A926D
:10501000AC85BD858C91A42DB52D8C9381E00E942B
:1050200064325A924A92AC85BD858D919C91A42D93
:10503000B52D8D939C9382E00E9464320E948F284C
:105040002C9687E00E946032089581E00E944433EC
:1050500081E00E944433AA85BB858C9180934702EE
:10506000A885B9858C9180934902AE81BF810C914E
:10507000013011F00C945228AA85BB850C9141E0B7
:10508000040FA8E4B2E00C93A885B9850C9141E027
:10509000040FAAE4B2E00C9384E0A881B9818C9358
:1050A0000C946028AA85BB858C9180934802A885C2
:1050B000B9858C9180934A0281E0A881B9818C9353
:1050C0000E94A722AC81BD818D919C91AFE4B2E09A
:1050D0008D939C930E94492D81E0AA81BB818C9382
:1050E000A881B9814C91AA81BB810C91041718F059
:1050F00011F00C94882892E0AFE5B2E00E941733DB
:10510000AA81BB818C918F5F8C9310F40C947028D2
:10511000C59A82E0481A8827580A2496089582E0A2
:105120000E94443382E00E94443382E00E94443370
:1051300082E00E94443382E00E94443382E00E9475
:10514000443382E00E94443381E00E94443381E092
:105150000E944433AC8DBD8D8C91AA81BB818C9310
:10516000AA8DBB8D8C91A881B9818C9380E090E051
:10517000A885B9858D939C93A88DB98D0D91112724
:10518000AC8DBD8D4D915527041B150BA889B98990
:105190000D931C93AE89BF890D911127AA8DBB8DEC
:1051A0004D915527041B150BAE85BF850D931C93A0
:1051B00081E090E0AC85BD858D939C9381E090E08B
:1051C000AA85BB858D939C93A889B9890D911C9163
:1051D000003050E015070CF402C00C9401298FEF49
:1051E0009FEFAC85BD858D939C93A889B9890D915E
:1051F0001C914FEF5FEF0E942F34A889B9890D935E
:105200001C93AE85BF850D911C91003050E01507B1
:105210000CF402C00C941E298FEF9FEFAA85BB856A
:105220008D939C93AE85BF850D911C914FEF5FEFE1
:105230000E942F34AE85BF850D931C93A889B98930
:105240004D915C91AE85BF850D911C91041715079A
:105250001CF011F00C94C62902E010E0A889B9896D
:105260004D915C910E942F34AE81BF810D931C93B0
:1052700002E010E0AE85BF854D915C910E942F3415
:10528000AC81BD810D931C93A88DB98D4C91AA81E1
:10529000BB810C91041711F40C94C4295A924A92C0
:1052A000AC81BD818C91A42DB52D8C9381E00E94A1
:1052B00064325A924A92AC81BD818C91A42DB52D55
:1052C0008C9381E00E9464325A924A92AA8DBB8DDF
:1052D0008C91A42DB52D8C9381E00E9464325A925A
:1052E0004A92AA8DBB8D8D919C91A42DB52D8D9345
:1052F0009C9382E00E9464320E942528289685E0D3
:105300000E946032AA81BB810C91AC85BD854C9115
:10531000040FAA81BB810C93A885B9850D911C91BE
:10532000AC81BD814D915C91040F151FA885B98595
:105330000D931C93A889B9894D915C91A885B98575
:105340000D911C91041715071CF011F00C94AA295B
:105350000C94C229A881B9810C91AA85BB854C9176
:10536000040FA881B9810C93A885B9850D911C9172
:10537000AE81BF814D915C91041B150BA885B98549
:105380000D931C930C9444290C945E2A02E010E0C7
:10539000AE85BF854D915C910E942F34AE81BF8157
:1053A0000D931C9302E010E0A889B9894D915C919E
:1053B0000E942F34AC81BD810D931C93AE89BF89AF
:1053C0004C91A881B9810C91041711F40C945E2AB8
:1053D0005A924A92AC81BD818C91A42DB52D8C93AB
:1053E00081E00E9464325A924A92AC81BD818C91D4
:1053F000A42DB52D8C9381E00E9464325A924A927A
:10540000AA8DBB8D8C91A42DB52D8C9381E00E942B
:1054100064325A924A92AA8DBB8D8D919C91A42D93
:10542000B52D8D939C9382E00E9464320E942528C2
:10543000289685E00E946032A881B9810C91AA85E6
:10544000BB854C91040FA881B9810C93A885B985BF
:105450000D911C91AC81BD814D915C91040F151F84
:10546000A885B9850D931C93AE85BF854D915C9140
:10547000A885B9850D911C91041715071CF011F032
:105480000C94442A0C945C2AAA81BB810C91AC85B3
:10549000BD854C91040FAA81BB810C93A885B98569
:1054A0000D911C91AE81BF814D915C91041B150B38
:1054B000A885B9850D931C930C94DE295A924A92C3
:1054C000AC81BD818C91A42DB52D8C9381E00E947F
:1054D00064325A924A92AC81BD818C91A42DB52D33
:1054E0008C9381E00E9464325A924A92AA8DBB8DBD
:1054F0008C91A42DB52D8C9381E00E9464325A9238
:105500004A92AA8DBB8D8D919C91A42DB52D8D9322
:105510009C9382E00E9464320E942528289685E0B0
:105520000E94603280E1481A8827580A62960895DE
:1055300081E00E94443381E00E94443381E00E9474
:10554000443381E00E94443381E00E94443382E08E
:105550000E94443381E00E94443381E00E9444333E
:1055600081E00E94443382E00E94443381E00E9443
:10557000443382E00E94443382E00E94443381E05D
:105580000E94443381E00E94443381E00E9444330E
:1055900081E00E944433AAA5BBA50C9144E0049F7E
:1055A000A8A1B9A10C92A8A1B9A18C9183508C9308
:1055B000A8A1B9A1AD90BB24A6E5B2E0AA0DBB1D80
:1055C0008C91AE8DBF8D8C93A8A1B9A18C918F5F6A
:1055D0008C93A8A1B9A1AD90BB24A6E5B2E0AA0D19
:1055E000BB1D8C91AE85BF858D9388278C93AE852E
:1055F000BF850C91AEA1BFA14C91049FAC8DBD8D18
:105600000C92A8A1B9A18C918F5F8C93A8A1B9A18C
:10561000AD90BB24A6E5B2E0AA0DBB1D8C91AA8D6E
:10562000BB8D8C93AA8DBB8D0C91A8A5B9A54C916F
:10563000049FAA8DBB8D0C92A8A1B9A18C918F5FFC
:105640008C93A8A1B9A1AD90BB24A6E5B2E0AA0DA8
:10565000BB1D8C91A88DB98D8C93A88DB98D0C91A3
:10566000AEA1BFA14C91049FA88DB98D0C9281E091
:10567000AC85BD858C93A8A9B9A90E947F38482F15
:10568000AC85BD850C91041718F011F00C94432DD6
:10569000AC85BD858C91E8A9F9A901E00A93AB8599
:1056A000BC850E946038AA85BB858C91AE89BF8974
:1056B0008D9388278C93AE89BF890D911C910A37F1
:1056C00050E0150718F011F00C94682B0C94CC2BBB
:1056D000AE89BF890D911C91043E50E0150711F071
:1056E0000C947A2B8FE790E0AE89BF898D939C93C1
:1056F0000C94CC2B063F50E0150711F00C94882B2E
:1057000080E890E0AE89BF898D939C930C94CC2B5C
:105710000C3F50E0150711F00C94962B81E890E0B7
:10572000AE89BF898D939C930C94CC2B043C50E0A4
:10573000150711F00C94A42B82E890E0AE89BF8984
:105740008D939C930C94CC2B063D50E0150711F0E3
:105750000C94B22B83E890E0AE89BF898D939C9323
:105760000C94CC2B0C3D50E0150711F00C94C02B81
:1057700084E890E0AE89BF898D939C930C94CC2BE8
:105780000F3D50E0150711F00C94CC2B85E890E00C
:10579000AE89BF898D939C93AE89BF890D911C9171
:1057A00040E250E0041B150BAE89BF890D931C939A
:1057B000AE85BF850D911C91AE89BF894D915C91DD
:1057C0000E942F34AE89BF890D931C93AC85BD8593
:1057D0000C9141E0041BAC89BD890C93AC89BD8957
:1057E0000C91AA8DBB8D4C91049FA7E4B2E00C9262
:1057F00000914702AEA5BFA54C91040FA7E4B2E00B
:105800000C93ACA5BDA58C9180934902AA8DBB8D4C
:105810000C9140914702040FA8E4B2E00C938091F0
:10582000480281508093480200914902A88DB98DA9
:105830004C91040FAAE4B2E00C9380914A0281508B
:1058400080934A020E94A72280E090E0A885B98553
:105850008D939C93AE85BF854D915C91A885B9854C
:105860000D911C910417150718F011F00C943A2DA6
:10587000AAA5BBA50C91013011F00C944D2CE2EEC1
:10588000FBE50E947137AE89BF898D919C91A1E59E
:10589000B2E00E941A370C945D2C023011F00C9487
:1058A0005D2CE2E1FFE50E947137AE89BF898D91E1
:1058B0009C91A1E5B2E00E941A3781E0AE81BF81E0
:1058C0008C93AEA1BFA14C91AE81BF810C91041706
:1058D00018F011F00C942F2DAE85BF854D915C9181
:1058E000A885B9850D911C910417150711F00C942A
:1058F0007C2C80E080935102A8A1B9A1AD90BB247B
:10590000A5E5B2E0AA0DBB1D0C91A8A1B9A1AD906F
:10591000BB24A3E5B2E0AA0DBB1D4C91041BAC81D6
:10592000BD810C93AC81BD810C91A8A5B9A54C910A
:10593000049FAC81BD810C9281E080935202AC81C6
:10594000BD814C9100915202041718F011F00C9493
:10595000C02CAAA1BBA18D919C91AFE4B2E08D9324
:105960009C930E94492D92E0AFE5B2E00E9417336C
:10597000A2E5B2E08C918F5F8C9310F40C949F2C75
:10598000AE8DBF8D0C9141E0041BAC81BD810C93A9
:10599000AC81BD818C91809352024091520200E013
:1059A000041718F011F00C94272D81E0AA81BB8117
:1059B0008C93A8A5B9A54C91AA81BB810C91041721
:1059C00018F011F00C941F2DA2E5B2E08C91A1E526
:1059D000B2E00E9427370E941D370C90082268947D
:1059E00009F4E894A881B981882780F98C93A8816B
:1059F000B9810C91013011F00C94082DACA1BDA11E
:105A00008D919C91AFE4B2E08D939C930C94102DFA
:105A1000AAA1BBA18D919C91AFE4B2E08D939C9320
:105A20000E94492D92E0AFE5B2E00E941733AA81AF
:105A3000BB818C918F5F8C9310F40C94D92C809146
:105A4000520281508093520210F00C94CD2CAE8102
:105A5000BF818C918F5F8C9310F40C94612CAE8974
:105A6000BF890E946832A885B9850E94683210F407
:105A70000C942A2CC59AAC85BD858C918F5F8C9334
:105A800010F40C943B2B85E1481A8827580AA296FB
:105A9000089580914F028093600298E0AFE4B2E0F5
:105AA0000E946C3480914F0280935F0208958CE2D3
:105AB00091E00E943533C4988BE490E00E94353326
:105AC000C5988BE490E00E943533C1988BE490E058
:105AD0000E943533C69A8BE490E00E943533C49A15
:105AE0008BE490E00E943533E8E9FBE50E947137D2
:105AF0000E94533281E080934702009147020532B1
:105B000018F011F00C94A62D0E945932ACE4B2E0CA
:105B10000E940A370E945332ACE4B2E00D911C910E
:105B2000003050E3150711F00C949C2D8BE490E0AD
:105B30000E9435330C949E2D0E94A92DA7E4B2E05B
:105B40008C918F5F8C9310F40C947D2DC59AC69820
:105B50000895C69AC59898E0ACE4B2E00E944C342F
:105B600091E0ACE4B2E00E94173398E0ACE4B2E01C
:105B70000E943F3491E0ACE4B2E00E941733C59A32
:105B8000C6980895C598AFEBB3E09C91AFE5B2E03D
:105B90000E941733C59A0895FDFDFDFD003000EF0A
:105BA00004EE041BFEFEFEFE90EF044A3F7F04EE6F
:105BB0000643003090EF83090008AF0B000A000590
:105BC0000006000700EF0CEE90EF8000B0EF0249F6
:105BD00000EF017F81E102E276E283E1018090EF54
:105BE00000000000000000000000040E0E0404008D
:105BF00004001B1B120000000000000A1F0A0A1FFD
:105C00000A00080E100C021C0400191902040813E3
:105C100013000814140815120D000C0C08000000E5
:105C20000000040808080808040008040404040428
:105C30000800000A0E1F0E0A00000004041F0404DE
:105C4000000000000000000C0C080000001F000015
:105C5000000000000000000C0C000001020408100D
:105C600000000E11131519110E00040C0404040495
:105C70000E000E11010608101F000E11010E011179
:105C80000E0002060A121F0202001F10101E011150
:105C90000E000608101E11110E001F010204080854
:105CA00008000E11110E11110E000E11110F01023C
:105CB0000C0000000C0C000C0C0000000C0C000C84
:105CC0000C08020408100804020000001F00001F56
:105CD000000008040201020408000E11010604007D
:105CE00004000E11171517100E000E11111F1111BF
:105CF00011001E11111E11111E000E111010101195
:105D00000E001E11111111111E001F10101E101077
:105D10001F001F10101E101010000E11101711116F
:105D20000F001111111F111111000E0404040404BD
:105D30000E000101010111110E00111214181412AC
:105D400011001010101010101F00111B151111114F
:105D5000110011191513111111000E11111111114A
:105D60000E001E11111E101010000E11111115122F
:105D70000D001E11111E121111000E11100E011135
:105D80000E001F0404040404040011111111111168
:105D90000E0011111111110A04001111151515151C
:105DA0000A0011110A040A1111001111110A040448
:105DB00004001E02040810101E000E08080808083F
:105DC0000E0000100804020100000E02020202028E
:105DD0000E00040A11000000000000000000000096
:105DE000001F0C0C04000000000000000E010F1149
:105DF0000F0010101E1111111E0000000E111011C5
:105E00000E0001010F1111110F0000000E111F10E3
:105E10000E000608081E0808080000000F11110FE8
:105E2000010E10101C1212121200040004040404CB
:105E30000400020006020202120C101012141814C0
:105E40001200040404040404060000001A151511CD
:105E5000110000001C121212120000000E1111118C
:105E60000E0000001E1111111E1000000F11111163
:105E70000F010000160908081C0000000E100E019A
:105E80000E0000081E08080A040000001212121674
:105E90000A0000001111110A040000001111151F61
:105EA0000A00000012120C12120000001212120E50
:105EB000041800001E020C101E000608081808082E
:105EC000060004040404040404000C020203020299
:105ED0000C0000000000000000000A000E010F117D
:105EE0000F000A000E1111110E000A0012121216F4
:105EF0000A000A0E111F111111000A0E11111111C1
:105F00000E000A11111111110E000C12121C1212A6
:105F10001C10000000000000000000000000000055
:105F2000000000183C3C3C181800181800000066DF
:105F30006666240000000000000000000000006C05
:105F40006CFE6C6C6CFE6C6C00000018187CC6C299
:105F5000C07C0686C67C18180000000000C2C60C73
:105F6000183066C60000000000386C6C3876DCCC57
:105F7000CC76000000181818300000000000000067
:105F800000000000000C183030303030180C0000D9
:105F900000000030180C0C0C0C0C18300000000035
:105FA000000000663CFF3C660000000000000000AE
:105FB0000018187E18180000000000000000000003
:105FC000000000181818300000000000000000FE5B
:105FD00000000000000000000000000000000000C1
:105FE0001818000000000002060C183060C0800085
:105FF0000000000000386CC6C6D6C6C66C3800006B
:1060000000000018387818181818187E00000000D2
:10601000007CC6060C183060C6FE00000000007C44
:10602000C606063C0606C67C00000000000C1C3CB0
:106030006CCCFE0C0C1E0000000000FEC0C0C0FCBA
:106040000606C67C00000000003860C0C0FCC6C662
:10605000C67C0000000000FEC6060C183030303050
:1060600000000000007CC6C6C67CC6C6C67C000018
:106070000000007CC6C6C67E06060C780000000044
:1060800000001818000000181800000000000000B0
:10609000181800000018183000000000000C18301C
:1060A00060C06030180C00000000000000007E009E
:1060B000007E000000000000006030180C060C1884
:1060C000306000000000007CC6C60C1818001818CC
:1060D00000000000007CC6C6DEDEDEDCC07C000006
:1060E00000000010386CC6C6FEC6C6C60000000020
:1060F00000FC6666667C666666FC00000000003C8C
:1061000066C2C0C0C0C2663C0000000000F86C66F9
:10611000666666666CF80000000000FE66626878DD
:10612000686266FE0000000000FE666268786860D3
:1061300060F000000000003C66C2C0C0DEC6663AE7
:106140000000000000C6C6C6C6FEC6C6C6C6000021
:106150000000003C181818181818183C000000001F
:10616000001E0C0C0C0C0CCCCC780000000000E6DF
:10617000666C6C786C6C66E60000000000F0606095
:106180006060606266FE0000000000C6EEFED6C6DB
:10619000C6C6C6C60000000000C6E6F6FEDECEC6D5
:1061A000C6C600000000007CC6C6C6C6C6C6C67C01
:1061B0000000000000FC6666667C606060F0000025
:1061C0000000007CC6C6C6C6C6D6DE7C0E00000037
:1061D00000FC6666667C6C6666E600000000007C7B
:1061E000C6C660380CC6C67C00000000007E7E5A21
:1061F00018181818183C0000000000C6C6C6C6C60D
:10620000C6C6C67C0000000000C6C6C6C6C6C66CB0
:1062100038100000000000C6C6C6C6D6D6FE6C6C9C
:106220000000000000C6C6C67C387CC6C6C600009A
:10623000000000666666663C1818183C0000000006
:1062400000FEC68C183060C2C6FE00000000003C94
:10625000303030303030303C000000000080C0E092
:1062600070381C0E060200000000003C0C0C0C0CE8
:106270000C0C0C3C000010386CC600000000000044
:10628000000000000000000000000000000000000E
:1062900000FF0030180C00000000000000000000AB
:1062A000000000000000780C7CCCCC7600000000E0
:1062B00000E06060786C6666667C000000000000AC
:1062C00000007CC6C0C0C67C00000000001C0C0C96
:1062D0003C6CCCCCCC7600000000000000007CC6FA
:1062E000FEC0C67C00000000001C3632307C30301E
:1062F0003078000000000000000076CCCCCC7C0C94
:10630000CC78000000E060606C76666666E60000AF
:1063100000000018180038181818183C0000000079
:10632000000606000E0606060666663C000000E053
:106330006060666C786C66E6000000000038181833
:1063400018181818183C0000000000000000ECFEAF
:10635000D6D6D6D60000000000000000DC666666D7
:10636000666600000000000000007CC6C6C6C67C51
:106370000000000000000000DC6666667C6060F0E3
:1063800000000000000076CCCCCC7C0C0C1E000081
:1063900000000000DC76666060F000000000000095
:1063A00000007CC6701CC67C00000000001030306D
:1063B000FC303030361C0000000000000000CCCC67
:1063C000CCCCCC760000000000000000C6C6C66C35
:1063D00038100000000000000000C6C6D6D6FE6CD3
:1063E0000000000000000000C66C38386CC60000D9
:1063F000000000000000C6C6C6C67E060C7800007D
:1064000000000000FECC183066FE00000000000E08
:10641000181818701818180E000000000018181826
:106420001818181818180000000000701818180E16
:10643000181818700000FF000000000000000000A5
:10644000000000FF000000480000780C7CCCCC76F7
:1064500000000000004800007CC6C6C6C67C0000E4
:10646000000000480000CCCCCCCCCC76000000442E
:106470000010386CC6C6FEC6C6C600000044007CCC
:10648000C6C6C6C6C6C6C67C0000004400C6C6C690
:10649000C6C6C6C6C67C000000000078CCCCF8CCCE
:1064A000CCCCF8C0C0C08E2E9F2E8BB7809300013D
:1064B0000895E82DF92D809100018BBF88940895EF
:1064C000481A8827580A0895480E8827581E0895A4
:1064D000ED91FC91EF5FFF4FFC93EE930895ED91EA
:1064E000FC91E150F040FC93EE93089509D00E9496
:1064F0002F3400FC10D0089503D01ED001F8F9CF3E
:106500000024E89457FF02C009D0689400F80BD02B
:1065100010F80124089502D009D0089550954095AF
:106520004F5F5F4F0895E89417FF08950095109509
:106530000F5F1F4F68940895352F242FE894452B43
:1065400011F468940895512F402F0027112780E1FE
:10655000440F551F001F111F021B130B416018F43D
:10656000020F131F4E7F8A9599F708958F938D918F
:106570008823E9F711978F910895A0E8BFE017D01D
:106580008D3049F0883079F03323C9F38D933A95F3
:1065900063FE43D0F4CF63FC03C03FD08AE03DD01C
:1065A00088278C93089539D011973395E8CF7F933E
:1065B0000F929F93AF93BF9380913F018823E1F3A4
:1065C000F89480913F018A9580933F0190913D011D
:1065D000A1E0B1E0A90F0024B01D8C9193959C33EC
:1065E00009F4992790933D017894BF91AF919F91C1
:1065F0000F907F910895A0E8BFE08D91882311F05E
:106600000CD0FBCF08950E940F36802D11F005D0DD
:10661000FACF08958DE001D08AE000909B0005FE3E
:10662000FCCF80939C0008953197F1F708950E9464
:1066300028338D910E942A339A95D9F70E942933E5
:106640000895B99ABB98C39ABA9A80E58DB908950E
:10665000089508958FB9779BFECF8FB10895689400
:1066600062F80895E89462F80895EF93FF93EE2797
:10667000E82BE92B31F0E0EAFFE03197F1F70197E1
:10668000D1F7FF91EF9108955A924A92480E8827C8
:10669000581E08958DE207FD8D938F2D881F802F42
:1066A000881F8F57082F6894F7F8802F87FF15C031
:1066B00080958395082F80E38D938EE28D93802FB4
:1066C000815228F080E38D9399279C930895442765
:1066D0000A95802F09F198D01FC0805230F09EE4B7
:1066E0009D9381E48D939D93EFCF4427DF92EF92AA
:1066F000FF920F938FE1801B11F0082F85D08BD074
:106700009EE29D930F91FF90EF90DF9044270395B9
:10671000003209F4D7CF2DD03F93E8EAF7E60E9484
:10672000713738E12F2D1E2D0D2DFF24EE24DD2491
:106730004427000F111F221FA8F42F923F920E949E
:106740000F36102C0E940F36202C0E940F36302C52
:106750000E940F363197410DD21CE31CF01C3F9074
:106760002F9001C0339631963A9519F73F9107D093
:10677000ADCFDD0CEE1CFF1C0A95D9F7089500275C
:1067800019E058D08F93802B11F0039501C08F91A1
:106790001A95B9F7802F882309F494CF8F91805DE3
:1067A0008D930A95D9F790CF0065CD1D80B2E60E86
:1067B00040597307A0ACB90350D6DC01286BEE003A
:1067C00094357700CA9A3B0065CD1D00B2E60E00F5
:1067D00059730700ACB90300D6DC01006BEE000072
:1067E000357700009A3B0000CD1D0000E60E00004A
:1067F00073070000B9030000DC010000EE00000098
:10680000770000003B000000F694E794D79447958A
:106810000A95D1F7089500270DD08F9303958F2DFA
:106820008E298D29842BC1F78F91805D8D930A95D8
:10683000D9F74ACF1F930F93002710E2440FDD1CB6
:10684000EE1CFF1C001F802F9AE0890B10F0082F10
:1068500043951A9599F7802F0F911F9108950F92E4
:10686000B801469F8001479F100D569F100D0F9055
:1068700008950E940F360D920020D9F708959030A8
:1068800051F000240D911C91000F111F001D9A95CD
:10689000D9F71C930E930895903051F00D911C91EF
:1068A0001695079508F410689A95D1F71C930E93E6
:1068B0000895903029F08C91880F9A95E9F78C9380
:1068C0000895903041F00D911C91000F111F9A9581
:1068D000E1F71C930E930895903041F00D911C91B7
:1068E000169507959A95E1F71C930E930895999143
:1068F0000027A90FB01F1197492F4A95FBB65E2FAD
:106900006F2FE89411274395203019F0D895802DEA
:1069100001C080818823E1F07C917723C9F078174A
:1069200059F40EF0042F139568941196319658F788
:106930008BB783958BBFE7CF112321F0411BA11BA0
:106940001127B10BE894E52FF62FFBBE1196DBCF94
:10695000882311F00027089508953DD09927112725
:106960008F2D880F80E8F82A802F881F08F41FEFEA
:1069700041F08F57082F07FD04C0003240F08FEF21
:1069800001C08827982FD82EE82EF82E09C08FE155
:10699000801B082FF694E794D79497950A95D1F722
:1069A000112351F09095D094E094F09481E0980FE9
:1069B0008827D81EE81EF81E0F2DFE2CED2CD92E90
:1069C0000895D094E094F09491E0D90E9927E91EAF
:1069D000F91E10950895D190E190F19001910895DC
:1069E00021913191419151910895102F90E8FF0C20
:1069F000001F0927990FF7941078652F90E8440F2E
:106A0000551F5927990F4795607800380895FF0C56
:106A100090E89027110F9795F794092F0895502F1C
:106A20002D2D3E2D4F2D612F08952DEC3CEC4CEC7F
:106A30005DE366270FC0CFDFF2DFDD24EE2490E8B0
:106A4000F92E0FE307C0CCDF05C02227332740E231
:106A500051E46627552351F1002381F1C6DF71F11E
:106A60001627005850580894050B18F407FD03C06A
:106A700025C007FD23C0469537952795F694E794E2
:106A8000D79422D0FF202AF0DD0CEE1CFF1C015011
:106A900073F09D2D969548F0DD203AF4EE202AF40F
:106AA00091E0D90E9927E91EF91EB1CF07C09FE7E3
:106AB000092FF92A9FEFD92EE92E0895DD24EE241F
:106AC000FF240027112708959F929924AA24BB240C
:106AD00088E1D216E306F40628F0D21AE30AF40A93
:106AE000089401C08894991CAA1CBB1CDD0CEE1CE8
:106AF000FF1C8A9571F7D92CEA2CFB2C9F900895E6
:106B000074DFE1F25038D1F216270058505808943B
:106B1000051F12F418F4CBCF08F0D0CF0BD0FF2014
:106B20002AF0BB0CDD1CEE1CFF1C71CF0F5F0BF4B9
:106B3000BECF6DCF9F929924AA24BB24992788E1C8
:106B4000990CAA1CBB1CDD1CEE1CFF1C30F4920E21
:106B5000A31EB41ED91EE91EF91E8A9589F79F90BF
:106B600008953EDF42DF503829F090E869270CC0D5
:106B70000AF045D04CCF5FE322273327442701C0DA
:106B80002FDF33DF5038B1F3003899F3902F951B86
:106B90008BF312F434D0FACF983118F02227332730
:106BA0004427983028F0232F342F44279850F9CFCA
:106BB000992329F04695379527959A95D9F7912FDE
:106BC000962742F014D0B0F6F794E794D7940F5F6D
:106BD0008BF66DCF10D051F008F4F3DEFF2052F2A7
:106BE000DD0CEE1CFF1C0150CBF761CF67CFD20E3E
:106BF000E31EF41E0895D21AE30AF40A0895DF9200
:106C0000EF92FF920F931F93D22EE32EF42E052FB7
:106C1000162F6F915F914F913F912F910895D895C5
:106C2000319628F48F938BB783958BBF8F9100207B
:106C30000895F5DF202DF3DF302DF1DF402DEFDF5C
:106C4000502D089507FB00680EF40F7757FB50682E
:106C50000EF45F7707FD02C057FF05C0D216E306AA
:106C6000F406050708952D153E054F0550070895B4
:106C70000E943233E89488278A938A931FDF112772
:106C80008D918032E9F31197BBD098F08D3229F4C1
:106C9000109511968C91B4D060F08E3229F4119633
:106CA0008C91AED008F446C022960E942F3381E02A
:106CB00008958C91A5D0D8F547D01196D0F70395BB
:106CC0008D919ED0E0F38E3229F48C9199D010F4FE
:106CD0001196FBCF853419F0853609F055C0119611
:106CE0008C918ED060F08D3219F08B3221F0DCCF98
:106CF00008800094088211968C9182D0A8F6805367
:106D0000898311968C917CD058F49981990F990FB1
:106D10000980900D990F8053890F8983873220F65F
:106D20008981988199230AF48195080F2DC08E32AC
:106D300089F611968C9164D068F606D018F01196F9
:106D40000A95F8CF1196C1CF4F2D3E2D2D2DDD0C7C
:106D5000EE1CFF1CA8F0DD0CEE1CFF1C88F0D20E10
:106D6000E31EF41E68F0DD0CEE1CFF1C48F080539F
:106D700009F06894D80E8827E81EF81E08F00895D8
:106D8000F42EE32ED22E089534D019F116F509838E
:106D900008E921D00695882787959F2D9F77980F22
:106DA000F92E0150000F110F07958981882379F082
:106DB0001AF48195898306C038DE89818A95898392
:106DC000D9F705C042DE89818A958983D9F7229651
:106DD000089574DEFCCF0DD041F0FF2032F00A950B
:106DE00031F0DD0CEE1CFF1CD2F788940895089456
:106DF000089500240D280E280F28002A0020089549
:106E0000803320F08A3310F408940895889408950C
:106E100091E005C092E003C094E001C098E028F43E
:106E20008F938BB783958BBF8F91F9DE0D929A95D7
:106E3000E1F70895E80FF91FEBCF91E0882321F0E7
:106E40008894991F8A95E9F7892F9095089588303D
:106E500018F011968850FBCF08952E2E3F2E9927BB
:106E600081918D3209F093958823D1F79A95E22D7F
:106E7000F32D112361F0091718F011F0101B01C058
:106E8000191B28F021F080E28D931A95E9F7808193
:106E90008D3219F48D93319604C0222311F08BE2C8
:106EA0008D93091738F031F0091B21F080E38D93A1
:106EB0000A95E9F781918D938823E1F7332351F007
:106EC000EA2FFB2F319633958E9182933A95E1F715
:106ED0008EE28C9308950F9301E00BBF0F9188947D
:106EE00008950F930027F9CF0F9302E0F6CF0F9389
:106EF00003E0F3CF7F930F93AF93BF938F939F9351
:106F00008FB78F93E89480913F010CE3081B29F41D
:106F100090919C000E942F3314C000913E01A1E08B
:106F2000B1E0772790919C00A00FB71F9C936894C5
:106F3000839580933F0103950C3309F40027009358
:106F40003E019D3011F40E943D028F918FBF9F91B1
:106F50008F91BF91AF910F917F9118956FB7F89472
:106F6000882793E08D939A95E9F76FBF0895040FF2
:106F7000151F261F371F0895000F111F221F331FD3
:106F8000089500951095209530950F5F1F4F2F4F56
:106F90003F4F0895019110810EC0019111912191EF
:106FA00030810BC00191108117FF05C03FEF2FEF1B
:106FB00004C0008111272227332737FF03C0E1DFF8
:106FC0008DE28D93CF93DF93CF92DF92EF92AA243D
:106FD000BB24CC24DD24EE2440E2CAE0DD2755E0CA
:106FE00093E38881890F87FD9F7083FD907F891BC4
:106FF00089935A95A9F7C0DFAA1CBB1CCC1CDD1CC9
:10700000EE1C4A9551F7E894EFE0FF2782910ED0ED
:10701000EB30E0F71EF068948A2D0CD088278D9312
:10702000EF90DF90CF90DF91CF910895982F8295C8
:1070300001D0892F8F70805D26F0803309F4089588
:1070400068948D93089500271127222733271DD098
:107050008A3328F4803318F005D015D0F9CF0EF418
:1070600090CF089580538F93402F512F622F732F0D
:1070700083DF82DF7CDF80DF8F919927080F191F64
:10708000291F391F08958D910895E894FCDF8032FF
:10709000E9F38B32D9F38930C9F38D3211F4689456
:1070A000F2CF089588278D93089581918D93882339
:1070B000E1F7089594E081918D939A95E1F7089511
:1070C00009919191992351F08A95D9F7319781913E
:1070D0008D930A9519F08823D1F70895E3CFFF9394
:1070E000881BF9E0001FFA9511F4FF910895881F9D
:1070F000841B18F4840F8894F5CF0894F3CF8FEF96
:1071000083959D919923E1F70895689401C0E894CF
:10711000AF93BF938D9116F0919103C00E940F36EB
:10712000902D891718F011F48823A1F7BF91AF9122
:107130000895E89463F80895689463F808954BDC23
:1071400080E003C048DC802F8078882321F0DF9224
:10715000EF92FF920F938F9348DC802F839512F468
:10716000ADDC1BC080958A95885E0AF415C08850F6
:107170001AF40CD0D92210C0DD2488501AF406D09D
:10718000E9220AC0EE2402D0F92206C09FEF8770E0
:10719000990F8A95EAF708953ADC8F918823D9F3FD
:1071A0005F914F913F912F910F934CDD0F9199F388
:1071B00090F302D05068E5CC5FE340E83327222704
:1071C00008954B59063D000000000000C04100003A
:1071D000C8410000E8410000004423DBF93D000005
:1071E00020410000A04100004842303A00003D002C
:1071F000303A31363D3100003A00206B6D2F680087
:10720000202020202020202020202020202020207E
:107210002020202000005374F672756E67212041F3
:1072200044584C206C6F77005374F672756E67216A
:10723000204144584C206869676800005374F67216
:10724000756E6721204779726F206C6F77005374D9
:10725000F672756E6721204779726F2068696768DA
:1072600000005374F672756E6721204675DF7363F4
:1072700068616C74657200005374616E64627900B9
:107280005600410050313A20000050323A200000B0
:1072900050333A20000050343A20000050353A2054
:0872A000000050363A20000006
:00000001FF
